:03000000026A1F72
:106A1F00758E1190000078FF79FFE4F0A3D9FBD8B1
:0D6A2F00F778FFE4F6D8FD75817F026A77E5
:106E12004401EC40490FDB4401E840C90FDB440167
:056E2200E43C8EFA358E
:064A9B009001CC1220285E
:104AA1009001D0E0FCA3E0FDA3E0FEA3E0FFEF2432
:104AB10069FFEE3474FEED34FFFDEC34FFFCEC12C3
:104AC1001B927BDF7A927986783D12196E9001D420
:104AD1001220287B007A0079C078419001D4E0FC53
:104AE100A3E0FDA3E0FEA3E0FF121A7712636E7B41
:104AF100007A0079C0784112196EC004C005C00661
:104B0100C0077F977E7E7DD57C409001D4E0F8A3DD
:104B1100E0F9A3E0FAA3E0FB12187DD003D002D0A4
:104B210001D000121879C004C005C006C0077F92E9
:104B31007E867DC07C419001CCE0F8A3E0F9A3E042
:104B4100FAA3E0FB12196EA804A905AA06AB07D0C7
:104B510007D006D005D00412187D9001DC12202860
:104B61009001D0E0FCA3E0FDA3E0FEA3E0FFEF2471
:104B710069FFEE3474FEED34FFFDEC34FFFCEC1202
:104B81001B929001CCE0F8A3E0F9A3E0FAA3E0FBCB
:104B910012187D7B307AE67958783D12196EA80497
:104BA100A905AA06AB077F817E0E7DBA7C43121848
:104BB100799001E4E0F8A3E0F9A3E0FAA3E0FB12A5
:104BC100196E9001D81220289001E8E0FCA3E0FDC5
:104BD100A3E0FEA3E0FF9001D8E0F8A3E0F9A3E091
:104BE100FAA3E0FB121B14602940279001D8E0FCD6
:104BF100A3E0FDA3E0FEA3E0FF9001E8E0F8A3E05D
:104C0100F9A3E0FAA3E0FB1218799001D812202849
:104C110080B69001E8E0FCA3E0FDA3E0FEA3E0FF85
:104C2100121B819001D8E0F8A3E0F9A3E0FAA3E018
:104C3100FB121B1450279001D8E0FCA3E0FDA3E078
:104C4100FEA3E0FF9001E8E0F8A3E0F9A3E0FAA3F6
:104C5100E0FB12187D9001D812202880B57F007EDC
:104C6100007D007C009001D8E0F8A3E0F9A3E0FA10
:104C7100A3E0FB121B14604840469001ECE0FCA34A
:104C8100E0FDA3E0FEA3E0FF9001D8E0F8A3E0F986
:104C9100A3E0FAA3E0FB121B1450259001D8E0FC1D
:104CA100A3E0FDA3E0FEA3E0FF9001E8E0F8A3E0AC
:104CB100F9A3E0FAA3E0FB1218799001D812202899
:104CC1007F007E007D007C009001D8E0F8A3E0F930
:104CD100A3E0FAA3E0FB121B14504B9001ECE0FCA3
:104CE100A3E0FDA3E0FEA3E0FF121B819001D8E049
:104CF100F8A3E0F9A3E0FAA3E0FB121B146027403C
:104D0100259001D8E0FCA3E0FDA3E0FEA3E0FF9025
:104D110001E8E0F8A3E0F9A3E0FAA3E0FB12187DB3
:104D21009001D81220289001D8E0FCA3E0FDA3E077
:104D3100FEA3E0FF125ABE7B247A0B7998783912D0
:104D4100196E9001DCE0F8A3E0F9A3E0FAA3E0FB1F
:104D510012187D9001E01220287B007A0079C0783A
:104D6100419001E0E0FCA3E0FDA3E0FEA3E0FF121F
:104D71001A7712636E7B007A0079C0784112196E3E
:104D8100A804A905AA06AB079001E0E0FCA3E0FD99
:094D9100A3E0FEA3E0FF12187973
:014D9A0022F6
:106E9F009001F71220289001F7E0FCA3E0FDA3E09A
:106EAF00FEA3E0FF12636EA804A905AA06AB079024
:106EBF0001F7E0FCA3E0FDA3E0FEA3E0FF121879C9
:106ECF009001E8E0F8A3E0F9A3E0FAA3E0FB1219C0
:026EDF006E2221
:060D470090015C1220285F
:100D4D0090015CE0FCA3E0FDA3E0FEA3E0FFEF2437
:100D5D0013FFEE342DFEED34FFFDEC34FFFCEC12F1
:100D6D001B92900160E0F8A3E0F9A3E0FAA3E0FB89
:100D7D0012187D9001641220287F8D7EA67D147C33
:100D8D003D900164E0F8A3E0F9A3E0FAA3E0FB12C3
:100D9D00196E7B807AF279BF783E12187D126E9FA4
:100DAD009001681220287F477E857D167C3D90013D
:100DBD0064E0F8A3E0F9A3E0FAA3E0FB12196E7B5F
:100DCD00937AA77984783E12187D126E9F90016CEC
:100DDD001220287F217EB47D0A7C3D900164E0F8CD
:100DED00A3E0F9A3E0FAA3E0FB12196E7BFF7ACD25
:100DFD007953783F12187D126E9F90017012202842
:100E0D007F4D7E6C7D337C3B900164E0F8A3E0F96F
:100E1D00A3E0FAA3E0FB12196E7B817A3D797E780F
:100E2D003F12187D126E9F9001741220287F007E54
:100E3D00007D007C40900170E0F8A3E0F9A3E0FA9A
:100E4D00A3E0FB12196EA804A905AA06AB07900131
:100E5D0068E0FCA3E0FDA3E0FEA3E0FF1218791209
:100E6D005AA87BF37A767914783F12196EC004C0B4
:100E7D0005C006C007900168E0FCA3E0FDA3E0FEFD
:100E8D00A3E0FF125AA87BE87AC179517840121974
:100E9D006EA804A905AA06AB077FB17E737D717C90
:100EAD0042121879D003D002D001D000121879C0A7
:100EBD0004C005C006C0077F007E007D007C409009
:100ECD000170E0F8A3E0F9A3E0FAA3E0FB12196EBC
:100EDD00125AA87B0C7A5979ED783E12196EA80436
:100EED00A905AA06AB07D007D006D005D004121865
:100EFD00799001781220287F007E007D007C409043
:100F0D000170E0F8A3E0F9A3E0FAA3E0FB12196E7B
:100F1D00C004C005C006C0077F007E007D007C4078
:100F2D00900168E0F8A3E0F9A3E0FAA3E0FB121941
:100F3D006ED003D002D001D000121879125AA87BBE
:100F4D00767A4F791E783D12196EC004C005C00621
:100F5D00C0077F007E007D007C40900168E0F8A313
:100F6D00E0F9A3E0FAA3E0FB12196E125AA87B9CDC
:100F7D007A5A79B6783D12196EA804A905AA06AB5E
:100F8D0007900178E0FCA3E0FDA3E0FEA3E0FF12D3
:100F9D001879A804A905AA06AB07D007D006D00575
:100FAD00D00412187DC004C005C006C0077F007EA6
:100FBD00007D007C40900170E0F8A3E0F9A3E0FA19
:100FCD00A3E0FB12196E900174E0F8A3E0F9A3E021
:100FDD00FAA3E0FB121879125AA87B687A96790465
:100FED00783D12196EA804A905AA06AB07D007D043
:100FFD0006D005D0041218799001781220287F00B0
:10100D007E007D007C40900170E0F8A3E0F9A3E044
:10101D00FAA3E0FB12196EA804A905AA06AB079066
:10102D000168E0FCA3E0FDA3E0FEA3E0FF12187948
:10103D00900174E0F8A3E0F9A3E0FAA3E0FB121825
:10104D007D125AA87BD87A2A79C1783C12196EC0C4
:10105D0004C005C006C0077F007E007D007C409067
:10106D000170E0F8A3E0F9A3E0FAA3E0FB12196E1A
:10107D00A804A905AA06AB07900168E0FCA3E0FD52
:10108D00A3E0FEA3E0FF121879125AA87B727A33FF
:10109D0079DC783C12196EA804A905AA06AB079055
:1010AD000178E0FCA3E0FDA3E0FEA3E0FF121879B8
:1010BD00D003D002D001D000121879C004C005C0F1
:1010CD0006C007900174E0F8A3E0F9A3E0FAA3E0ED
:1010DD00FB900168E0FCA3E0FDA3E0FEA3E0FF129E
:1010ED001879125AA87B307A4C79A6783C12196E71
:1010FD00A804A905AA06AB07D007D006D005D004D1
:10110D00121879900178122028900170E0FCA3E06C
:10111D00FDA3E0FEA3E0FF125AA87B0B7AD2798CD7
:10112D00783C12196E900178E0F8A3E0F9A3E0FA8B
:10113D00A3E0FB12187DC004C005C006C0079001D6
:10114D0074E0FCA3E0FDA3E0FEA3E0FF900168E0E6
:10115D00F8A3E0F9A3E0FAA3E0FB12187D125AA858
:10116D007B697AE37988783C12196EA804A905AADF
:10117D0006AB07D007D006D005D00412187D90011C
:10118D00781220287F007E007D007C4090016CE06D
:10119D00F8A3E0F9A3E0FAA3E0FB12196EA804A9E5
:1011AD0005AA06AB07900168E0FCA3E0FDA3E0FEF5
:1011BD00A3E0FF121879125AA87BF97A4E794C7870
:1011CD003C12196EC004C005C006C007900174E042
:1011DD00FCA3E0FDA3E0FEA3E0FF125AA87BCD7AAD
:1011ED00AF79E6783B12196EA804A905AA06AB07DC
:1011FD00D007D006D005D00412187DC004C005C09C
:10120D0006C0077F007E007D007C40900170E0F8F5
:10121D00A3E0F9A3E0FAA3E0FB12196E900174E0CC
:10122D00F8A3E0F9A3E0FAA3E0FB12187D125AA887
:10123D007BBC7A5779AD783B12196EA804A905AA23
:10124D0006AB07D007D006D005D00412187DC00418
:10125D00C005C006C0077F007E007D807C409001E8
:10126D0070E0F8A3E0F9A3E0FAA3E0FB12196EA871
:10127D0004A905AA06AB07900168E0FCA3E0FDA355
:10128D00E0FEA3E0FF121879125AA87B4E7AB479CA
:10129D00AB783B12196EA804A905AA06AB07D007B7
:1012AD00D006D005D00412187990017C1220287F29
:1012BD00007E007D007C40900170E0F8A3E0F9A372
:1012CD00E0FAA3E0FB12196EA804A905AA06AB0764
:1012DD00900168E0FCA3E0FDA3E0FEA3E0FF12187F
:1012ED0079900174E0F8A3E0F9A3E0FAA3E0FB1212
:1012FD001879125AA87BA97A6A7982783B12196EED
:10130D0090017CE0F8A3E0F9A3E0FAA3E0FB12184A
:10131D007DC004C005C006C0077F007E007D407CF7
:10132D0040900168E0F8A3E0F9A3E0FAA3E0FB1216
:10133D00196E125AA87B9C7ADC796F783B12196E64
:10134D00A804A905AA06AB07D007D006D005D0047E
:10135D00121879C004C005C006C0077F007E007D4D
:10136D00807C40900170E0F8A3E0F9A3E0FAA3E0DF
:10137D00FB12196EC004C005C006C0077F007E00B9
:10138D007D007C40900168E0F8A3E0F9A3E0FAA3AA
:10139D00E0FB12196ED003D002D001D000121879E3
:1013AD00125AA87BCA7A547941783B12196EA80457
:1013BD00A905AA06AB07D007D006D005D004121890
:1013CD007990017C1220287F007E007D007C40906A
:1013DD000170E0F8A3E0F9A3E0FAA3E0FB12196EA7
:1013ED00C004C005C006C0077F007E007D407C4064
:1013FD00900168E0F8A3E0F9A3E0FAA3E0FB12196D
:10140D006ED003D002D001D000121879125AA87BE9
:10141D00457A2F7923783B12196EC004C005C0069A
:10142D00C007900174E0FCA3E0FDA3E0FEA3E0FF84
:10143D00900170E0F8A3E0F9A3E0FAA3E0FB121825
:10144D007D125AA87B147A5C792C783B12196EA800
:10145D0004A905AA06AB0790017CE0FCA3E0FDA35F
:10146D00E0FEA3E0FF121879A804A905AA06AB07B0
:10147D00D007D006D005D00412187DC004C005C019
:10148D0006C0077F007E007D007C40900170E0F873
:10149D00A3E0F9A3E0FAA3E0FB12196E900168E056
:1014AD00F8A3E0F9A3E0FAA3E0FB12187D90017414
:1014BD00E0F8A3E0F9A3E0FAA3E0FB121879125AC1
:1014CD00A87BA67AD57910783B12196EA804A905C8
:1014DD00AA06AB07D007D006D005D004121879C0E4
:1014ED0004C005C006C0077F007E007D007C4090D3
:1014FD000170E0F8A3E0F9A3E0FAA3E0FB12196E86
:10150D00C004C005C006C0077F007E007D007C4082
:10151D0090016CE0F8A3E0F9A3E0FAA3E0FB121947
:10152D006ED003D002D001D000121879125AA87BC8
:10153D00B37A7B79F2783A12196EA804A905AA0636
:10154D00AB07D007D006D005D00412187D90017CD2
:10155D001220287F007E007D007C4090016CE0F819
:10156D00A3E0F9A3E0FAA3E0FB12196E900168E085
:10157D00F8A3E0F9A3E0FAA3E0FB12187DC004C0C4
:10158D0005C006C0077F007E007D007C4090017085
:10159D00E0F8A3E0F9A3E0FAA3E0FB12196EA804AA
:1015AD00A905AA06AB07D007D006D005D00412189E
:1015BD0079125AA87B047AAD79C0783A12196EC0A7
:1015CD0004C005C006C0077F007E007D007C4090F2
:1015DD000174E0F8A3E0F9A3E0FAA3E0FB12196EA1
:1015ED00C004C005C006C0077F007E007D007C40A2
:1015FD00900170E0F8A3E0F9A3E0FAA3E0FB121963
:10160D006ED003D002D001D000121879125AA87BE7
:10161D00A37A0679D378BA12196EA804A905AA0679
:10162D00AB07D007D006D005D00412187DC004C07A
:10163D0005C006C0077F007E007D807C4090017054
:10164D00E0F8A3E0F9A3E0FAA3E0FB12196E125A39
:10165D00A87B4B7A1F79BA783A12196EA804A9059E
:10166D00AA06AB07D007D006D005D004121879C052
:10167D0004C005C006C0077F007E007D007C409041
:10168D000170E0F8A3E0F9A3E0FAA3E0FB12196EF4
:10169D00C004C005C006C0077F007E007D007C40F1
:1016AD00900168E0F8A3E0F9A3E0FAA3E0FB1219BA
:1016BD006ED003D002D001D000121879900174E0E1
:1016CD00F8A3E0F9A3E0FAA3E0FB12187D125AA8E3
:1016DD007BA97A3079B6783A12196EA804A905AAB1
:1016ED0006AB07D007D006D005D00412187D9001A7
:1016FD00801220287F007E007D807C40900170E06C
:10170D00F8A3E0F9A3E0FAA3E0FB12196EA804A96F
:10171D0005AA06AB07900168E0FCA3E0FDA3E0FE7F
:10172D00A3E0FF121879900174E0F8A3E0F9A3E0AB
:10173D00FAA3E0FB12187D125AA87B3B7AAA799A7C
:10174D00783A12196EA804A905AA06AB0790018074
:10175D00E0FCA3E0FDA3E0FEA3E0FF121879C004B6
:10176D00C005C006C0077F007E007D007C40900153
:10177D0070E0F8A3E0F9A3E0FAA3E0FB12196EC044
:10178D0004C005C006C0077F007E007D007C409030
:10179D000168E0F8A3E0F9A3E0FAA3E0FB12196EEB
:1017AD00A804A905AA06AB07D007D006D005D0041A
:1017BD0012187D125AA87B247A0B7998783A12194F
:1017CD006EA804A905AA06AB07D007D006D005D090
:1017DD0004121879C004C005C006C0077F007E0042
:1017ED007D007C40900168E0F8A3E0F9A3E0FAA346
:1017FD00E0FB12196E900174E0F8A3E0F9A3E0FA92
:10180D00A3E0FB121879125AA87BE07A2D79907813
:10181D003A12196EA804A905AA06AB07D007D0067F
:10182D00D005D00412187990018012202890017CE7
:10183D00E0FCA3E0FDA3E0FEA3E0FF900178E0F85B
:10184D00A3E0F9A3E0FAA3E0FB12187D900180E07C
:10185D00F8A3E0F9A3E0FAA3E0FB12187D7B487A28
:08186D005179C7784512196E8C
:011875002250
:0B2B9E00900122EBF0A3EAF0A3E9F0A5
:102BA900900128E0FCA3E0FDA3E0FEA3E0FFEC1206
:102BB9001B927B007A81798878C612187D90012C46
:102BC900E0F8A3E0F9A3E0FAA3E0FB12187D900175
:102BD900301220287F0A7EEB7D157C3D900130E084
:102BE900F8A3E0F9A3E0FAA3E0FB12196E7B7F7A60
:102BF9004F7940783F12187D126E9F900134122050
:102C0900287F8C7EA67D147C3D900130E0F8A3E0FE
:102C1900F9A3E0FAA3E0FB12196E7B367A90795298
:102C2900783F12187D126E9F9001381220287F4D2F
:102C39007E6C7D337C3B900130E0F8A3E0F9A3E0A2
:102C4900FAA3E0FB12196E7B857AEA797E783F1246
:102C5900187D126E9F90013C1220287F217EB47D41
:102C69000A7C3D900130E0F8A3E0F9A3E0FAA3E083
:102C7900FB12196E7BD37A697979783F12187D1224
:102C89006E9F9001401220287F477E857D167C3DEE
:102C9900900130E0F8A3E0F9A3E0FAA3E0FB1219F0
:102CA9006E7B9F7A027900783D12187D126E9F9093
:102CB90001441220287F007E007D007C4090014065
:102CC900E0F8A3E0F9A3E0FAA3E0FB12196E125AA7
:102CD900BE7BB07A727928783F12196EC004C0059C
:102CE900C006C007900138E0FCA3E0FDA3E0FEA305
:102CF900E0FF125ABE7B7D7A3F79C9784012196E7E
:102D0900A804A905AA06AB07D007D006D005D004A8
:102D190012187DC004C005C006C0077F007E007D73
:102D2900007C40900140E0F8A3E0F9A3E0FAA3E0B9
:102D3900FB12196EA804A905AA06AB07900138E091
:102D4900FCA3E0FDA3E0FEA3E0FF121879125ABE2E
:102D59007B6F7A1279A3783F12196EA804A905AA84
:102D690006AB07D007D006D005D004121879C004E5
:102D7900C005C006C00790013CE0FCA3E0FDA3E04C
:102D8900FEA3E0FF125ABE7BC97A76793E783E12DD
:102D9900196EA804A905AA06AB07D007D006D00565
:102DA900D0041218799001E4E0F8A3E0F9A3E0FA5D
:102DB900A3E0FB12196E900134E0F8A3E0F9A3E057
:102DC900FAA3E0FB12187D900148122028900148CF
:102DD900E0FCA3E0FDA3E0FEA3E0FFC004C005C042
:102DE90006C0077F007E007D007C40900144E0F82A
:102DF900A3E0F9A3E0FAA3E0FB12196E125ABE7B15
:102E0900D57A7879E9783D12196EC004C005C006F3
:102E1900C0077F007E007D007C40900138E0F8A368
:102E2900E0F9A3E0FAA3E0FB12196E125ABE7BD1B6
:102E39007A22795B783E12196ED003D002D001D084
:102E490000121879C004C005C006C0077F007E00C3
:102E59007D007C40900140E0F8A3E0F9A3E0FAA3EB
:102E6900E0FB12196EC004C005C006C0077F007ED2
:102E7900007D007C40900138E0F8A3E0F9A3E0FA76
:102E8900A3E0FB12196ED003D002D001D0001218B2
:102E990079125ABE7BFC7AA97971783D12196EA80C
:102EA90004A905AA06AB07D007D006D005D004129D
:102EB9001879C004C005C006C0077F007E007D00E8
:102EC9007C40900140E0F8A3E0F9A3E0FAA3E0FB1D
:102ED90012196EC004C005C006C00790013CE0FC91
:102EE900A3E0FDA3E0FEA3E0FF900138E0F8A3E032
:102EF900F9A3E0FAA3E0FB12187DD003D002D001B8
:102F0900D000121879125ABE7BD57A787969783D42
:102F190012196EA804A905AA06AB07D007D006D0D6
:102F290005D0041218799001E4E0F8A3E0F9A3E0D0
:102F3900FAA3E0FB12196EA804A905AA06AB07D0EB
:102F490007D006D005D00412187D90014812202818
:102F59007F007E007D007C40900140E0F8A3E0F90D
:102F6900A3E0FAA3E0FB12196E125ABE7BE37AC7FB
:102F79007928783F12196EC004C005C006C00790B1
:102F89000138E0FCA3E0FDA3E0FEA3E0FF125ABE76
:102F99007B9E7A5E79C7784012196EA804A905AAA2
:102FA90006AB07D007D006D005D00412187DC0049F
:102FB900C005C006C0077F007E007D007C409001EF
:102FC90040E0F8A3E0F9A3E0FAA3E0FB12196EA828
:102FD90004A905AA06AB07900138E0FCA3E0FDA30C
:102FE900E0FEA3E0FF121879125ABE7BE57AD07988
:102FF900A2783F12196EA804A905AA06AB07D00743
:10300900D006D005D0041218799001E4E0F8A3E0C5
:10301900F9A3E0FAA3E0FB12196E900144E0F8A3CA
:10302900E0F9A3E0FAA3E0FB12187D90014C12200D
:10303900287F007E007D007C40900140E0F8A3E0FD
:10304900F9A3E0FAA3E0FB12196EA804A905AA06E0
:10305900AB07900144E0FCA3E0FDA3E0FEA3E0FF81
:10306900121879125ABE7B067A817915783E12199F
:103079006EC004C005C006C00790014CE0FCA3E087
:10308900FDA3E0FEA3E0FF125ABE7BA67A9B79A4BA
:10309900784012196ED003D002D001D000121879ED
:1030A9009001E4E0F8A3E0F9A3E0FAA3E0FB121928
:1030B9006E900150122028900148E0FCA3E0FDA386
:1030C900E0FEA3E0FF125ABEC004C005C006C00757
:1030D900900150E0FCA3E0FDA3E0FEA3E0FF125A3B
:1030E900A8A804A905AA06AB07D007D006D005D021
:1030F9000412196E7B327AAF79CB783E12196EC001
:1031090004C005C006C007900150E0FCA3E0FDA380
:10311900E0FEA3E0FF125ABE7BDB7ADE796A783FD4
:1031290012196EA804A905AA06AB07D007D006D0C4
:1031390005D00412187D900125E0FBA3E0FAA3E075
:10314900F9121FB6900125E0FBA3E0FAA3E0F912FA
:103159001F96900125E0FBA3E0FAA3E0F9122008ED
:1031690012196EA804A905AA06AB077F007E007D87
:10317900807C3F1218791268309000EA122028905A
:103189000125E0FBA3E0FAA3E0F9121F96126ABC3D
:10319900900125E0FBA3E0FAA3E0F9121FB6900124
:1031A90048E0FCA3E0FDA3E0FEA3E0FF125AA8C09B
:1031B90004C005C006C007900150E0FCA3E0FDA3D0
:1031C900E0FEA3E0FF125AA8A804A905AA06AB07C6
:1031D900D007D006D005D00412196EC004C005C0AE
:1031E90006C007900125E0FBA3E0FAA3E0F9121F4E
:1031F90096125AA8A804A905AA06AB07D007D006B3
:10320900D005D004121A7790015412202890014851
:10321900E0FCA3E0FDA3E0FEA3E0FF125ABEC00458
:10322900C005C006C007900150E0FCA3E0FDA3E083
:10323900FEA3E0FF125AA8A804A905AA06AB07D065
:1032490007D006D005D00412196E7BDB7ADE796AC5
:10325900783F12196EC004C005C006C0079001501E
:10326900E0FCA3E0FDA3E0FEA3E0FF125ABE7B321F
:103279007AAF79CB783E12196EA804A905AA06ABD4
:1032890007D007D006D005D004121879C004C005AC
:10329900C006C007900125E0FBA3E0FAA3E0F912FC
:1032A9001F96125AA8A804A905AA06AB07D007D0E9
:1032B90006D005D004121A779001581220289001DF
:1032C90058E0FCA3E0FDA3E0FEA3E0FFC004C005B5
:1032D900C006C007900154E0FCA3E0FDA3E0FEA3F3
:1032E900E0FF9000EA122028D007D006D005D004CC
:1032F900126ABC900122E0FBA3E0FAA3E0F9121FD5
:10330900B6900122E0FBA3E0FAA3E0F9121F967B35
:10331900007A0079007800121B146030402E900169
:1033290022E0FBA3E0FAA3E0F9C003C002C0011246
:103339001F969001E8E0F8A3E0F9A3E0FAA3E0FB07
:1033490012187DD001D002D003121FB6900122E0DD
:10335900FBA3E0FAA3E0F9121F969001E8E0F8A3B5
:10336900E0F9A3E0FAA3E0FB121B14502E9001220E
:10337900E0FBA3E0FAA3E0F9C003C002C001121FF9
:10338900969001E8E0F8A3E0F9A3E0FAA3E0FB12C4
:0B3399001879D001D002D003121FB63B
:0133A4002206
:0B46D3009001AAEBF0A3EAF0A3E9F0CD
:1046DE009001B0E0FCA3E0FDA3E0FEA3E0FFEC122E
:1046EE001B927B007A81798878C612187D9001B46E
:1046FE00E0F8A3E0F9A3E0FAA3E0FB12187D7B003B
:10470E007AAD790E7847121A779001B81220287F69
:10471E00A67EFE7DC77C429001B8E0F8A3E0F9A327
:10472E00E0FAA3E0FB12196E7B917AEA797E783F6C
:10473E0012187D126E9F9001BC1220287F117E23CD
:10474E007D5F7C379001B8E0F8A3E0F9A3E0FAA30F
:10475E00E0FB12196EA804A905AA06AB077F507ECE
:10476E00AC7DAE7C3B121879126E9FC004C005C0A2
:10477E0006C0079001BCE0FCA3E0FDA3E0FEA3E0B1
:10478E00FF125ABEA804A905AA06AB07D007D00689
:10479E00D005D00412196EC004C005C006C0077F34
:1047AE00187E017DC87C429001B8E0F8A3E0F9A321
:1047BE00E0FAA3E0FB12196E7B327AE47946783F79
:1047CE0012187D126E9FA804A905AA06AB07D00782
:1047DE00D006D005D00412187DC004C005C006C096
:1047EE00077F007E007D007C409001BCE0F8A3E0D6
:1047FE00F9A3E0FAA3E0FB12196E125ABE7B0C7AF3
:10480E00347969783812196EA804A905AA06AB077F
:10481E00D007D006D005D00412187D9001C012200A
:10482E00287F147E6A7D177C389001B8E0F8A3E0EB
:10483E00F9A3E0FAA3E0FB12196EA804A905AA06D3
:10484E00AB077F6D7E6A7D857C3D121879126E9F57
:10485E009001C41220289001C0E0FCA3E0FDA3E06B
:10486E00FEA3E0FF125AFAC004C005C006C00790AE
:10487E0001C4E0FCA3E0FDA3E0FEA3E0FF125AA8F2
:10488E00A804A905AA06AB07D007D006D005D00408
:10489E0012196E125C089001AAE0FBA3E0FAA3E0E5
:1048AE00F9121FB69001E8E0F8A3E0F9A3E0FAA32D
:1048BE00E0FB9001C0E0FCA3E0FDA3E0FEA3E0FF5F
:1048CE00121A7712636E9001E8E0F8A3E0F9A3E004
:1048DE00FAA3E0FB12196EA804A905AA06AB07906D
:1048EE0001C0E0FCA3E0FDA3E0FEA3E0FF121879F7
:1048FE009001C81220287F007E007DC07C3F900171
:10490E00ECE0F8A3E0F9A3E0FAA3E0FB12196E9035
:10491E0001C8E0F8A3E0F9A3E0FAA3E0FB121B1430
:10492E00505A7F007E007D007C3F9001ECE0F8A3A2
:10493E00E0F9A3E0FAA3E0FB12196E9001C8E0F8CB
:10494E00A3E0F9A3E0FAA3E0FB121B14402E9001A2
:10495E00AAE0FBA3E0FAA3E0F9C003C002C0011273
:10496E001F969001ECE0F8A3E0F9A3E0FAA3E0FBB8
:10497E0012187DD001D002D003121FB69001AAE00A
:10498E00FBA3E0FAA3E0F9C003C002C001121F9618
:10499E00C004C005C006C0079001AAE0FBA3E0FA60
:1049AE00A3E0F9121F969001E8E0F8A3E0F9A3E066
:1049BE00FAA3E0FB121A7712636E9001E8E0F8A3F7
:1049CE00E0F9A3E0FAA3E0FB12196EA804A905AA68
:1049DE0006AB07D007D006D005D004121879D00147
:1049EE00D002D003121FB69001C0E0FCA3E0FDA3DD
:1049FE00E0FEA3E0FF125ABEC004C005C006C00709
:104A0E009001C4E0FCA3E0FDA3E0FEA3E0FF125A78
:104A1E00BEA804A905AA06AB07D007D006D005D0BC
:104A2E000412196E9001ADE0FBA3E0FAA3E0F912B7
:104A3E001FB69001ADE0FBA3E0FAA3E0F9121F96BA
:104A4E009001ADE0FBA3E0FAA3E0F91220081219E1
:104A5E006EA804A905AA06AB077F007E007D807CA8
:104A6E003F1218791268309000EA1220289001AD9A
:104A7E00E0FBA3E0FAA3E0F9121F96126ABC9001C4
:0C4A8E00ADE0FBA3E0FAA3E0F9121FB6B4
:014A9A0022F9
:0B33A500900184EBF0A3EAF0A3E9F034
:1033B0007F927E0A7D867C3E90018AE0F8A3E0F948
:1033C000A3E0FAA3E0FB12196E90018EE0F8A3E0EF
:1033D000F9A3E0FAA3E0FB121879900196122028D5
:1033E0007F007E007D007C00900196E0F8A3E0F96C
:1033F000A3E0FAA3E0FB121B145027900196E0FC17
:10340000A3E0FDA3E0FEA3E0FF9001E8E0F8A3E065
:10341000F9A3E0FAA3E0FB12187D90019612202890
:1034200080489001E8E0FCA3E0FDA3E0FEA3E0FFFC
:10343000900196E0F8A3E0F9A3E0FAA3E0FB121BE9
:103440001460274025900196E0FCA3E0FDA3E0FE78
:10345000A3E0FF9001E8E0F8A3E0F9A3E0FAA3E01D
:10346000FB121879900196122028900196E0F8A39B
:10347000E0F9A3E0FAA3E0FB900020E0FCA3E0FD6C
:10348000A3E0FEA3E0FF1218799000181220289004
:103490000018E0FCA3E0FDA3E0FEA3E0FF125AA8A1
:1034A000C004C005C006C00790001CE0FCA3E0FDFE
:1034B000A3E0FEA3E0FF125AA8A804A905AA06AB40
:1034C00007D007D006D005D00412196EC004C0057D
:1034D000C006C007900192E0FCA3E0FDA3E0FEA3BC
:1034E000E0FF125AA8A804A905AA06AB07D007D086
:1034F00006D005D00412196EC004C005C006C0076E
:1035000090001CE0FCA3E0FDA3E0FEA3E0FF125A44
:10351000BEC004C005C006C007900192E0FCA3E055
:10352000FDA3E0FEA3E0FF125ABEA804A905AA0667
:10353000AB07D007D006D005D00412196EA804A995
:1035400005AA06AB07D007D006D005D00412187D17
:1035500090019A12202890019AE0FCA3E0FDA3E0DC
:10356000FEA3E0FF90019AE0F8A3E0F9A3E0FAA33C
:10357000E0FB12196EA804A905AA06AB077F007E1E
:10358000007D807C3F12187912683090019E1220D5
:103590002890019AE0FCA3E0FDA3E0FEA3E0FFC0B9
:1035A00004C005C006C00790019EE0FCA3E0FDA397
:1035B000E0FEA3E0FF9000EA122028D007D006D05A
:1035C00005D004126ABC900187E0FBA3E0FAA3E0F7
:1035D000F9121FB6900187E0FBA3E0FAA3E0F9120D
:1035E0001F96125AA8C004C005C006C007900187E4
:1035F000E0FBA3E0FAA3E0F9121F96125ABED00333
:10360000D002D001D000121A77C004C005C006C095
:103610000790001CE0FCA3E0FDA3E0FEA3E0FF1286
:103620005AA8C004C005C006C00790001CE0FCA357
:10363000E0FDA3E0FEA3E0FF125ABED003D002D00B
:1036400001D000121A77A804A905AA06AB07D00773
:10365000D006D005D00412196EC004C005C006C043
:1036600007900187E0FBA3E0FAA3E0F9121F96128E
:103670005AA8C004C005C006C00790001CE0FCA307
:10368000E0FDA3E0FEA3E0FF125AA8A804A905AA42
:1036900006AB07D007D006D005D00412196EC004BF
:1036A000C005C006C007900192E0FCA3E0FDA3E0C6
:1036B000FEA3E0FF125ABED003D002D001D0001208
:1036C0001A77D003D002D001D0001218799001A649
:1036D000122028900192E0FCA3E0FDA3E0FEA3E00D
:1036E000FF125AA8C004C005C006C00790001CE025
:1036F000FCA3E0FDA3E0FEA3E0FF125AA8A804A9E2
:1037000005AA06AB07D007D006D005D00412196E63
:10371000C004C005C006C007900018E0FCA3E0FD8F
:10372000A3E0FEA3E0FF125AA8A804A905AA06ABCD
:1037300007D007D006D005D00412196EC004C0050A
:10374000C006C007900192E0FCA3E0FDA3E0FEA349
:10375000E0FF125ABEC004C005C006C00790001C9E
:10376000E0FCA3E0FDA3E0FEA3E0FF125ABEA80424
:10377000A905AA06AB07D007D006D005D0041219B8
:103780006EA804A905AA06AB07D007D006D005D0BD
:103790000412187D9001A2122028900192E0FCA34F
:1037A000E0FDA3E0FEA3E0FF125AA8C004C005C0DC
:1037B00006C007900018E0FCA3E0FDA3E0FEA3E034
:1037C000FF125ABEA804A905AA06AB07D007D00667
:1037D000D005D00412196EC004C005C006C0079001
:1037E00001A2E0FCA3E0FDA3E0FEA3E0FF9001A2A4
:1037F000E0F8A3E0F9A3E0FAA3E0FB12196EA80435
:10380000A905AA06AB077F007E007D807C3F1218C9
:1038100079126830A804A905AA06AB07D007D0061C
:10382000D005D004121A779001A21220289001A28C
:10383000E0FCA3E0FDA3E0FEA3E0FFC004C005C0E0
:1038400006C0079001A6E0FCA3E0FDA3E0FEA3E014
:10385000FF9000EA122028D007D006D005D004122D
:103860006ABC900184E0FBA3E0FAA3E0F9121FB662
:10387000900184E0FBA3E0FAA3E0F9121F967B001D
:103880007A0079007800121B146030402E90018479
:10389000E0FBA3E0FAA3E0F9C003C002C001121FDD
:1038A000969001E8E0F8A3E0F9A3E0FAA3E0FB12A8
:0B38B000187DD001D002D003121FB61B
:0138BB0022EA
:10678000323B171C0205006400640001000007A3EF
:1067900000870384006407080384068205690007F4
:1067A00000020009003B003B0017001C000C0063C6
:1067B00000C700C70002000A0E0F03840E0F0384F7
:1067C0000E0F07080E0F070800080007000E000054
:1067D00000000000000100010000000100010000B5
:1067E00000000000000000000000000000000000A9
:1067F0000000000000000000000000030000000393
:106800000002000300020003000300020003000274
:106810000003000000030001000300020003000267
:0C6820000003000300020003000200035C
:066E2700C119C11BC11AD4
:106BF3009000127432F0900013743BF09000147400
:106C030017F0900015741CF09000167402F09000B9
:106C1300177405F0125095757900757A00D3E57AEB
:106C2300940EE57964809480503CE57A25E0FFE595
:106C33007933FE74862FF58274673EF583E493FC03
:106C4300740193FDE57A25E0FFE57933FE74242F83
:106C5300F58274003EF583ECF0A3EDF0057AE57A56
:106C63007002057980B712519990006AE4F0A3E4A9
:106C7300F090006CE4F0A3E4F090006EE4F0A3E481
:056C8300F01251BB22DC
:103DAC00900041E0F574D3E57464809482400BC3B9
:103DBC00E574648094865002C219E5A064FFFFEF9D
:103DCC005407F576E5766006C29CC2988002D29CB8
:103DDC00E5765406FFEF60270578E578D3940A4022
:103DEC000F75750AC3E57464809486500375780A60
:103DFC00E578D39414400E75756475781480067547
:103E0C007800757501AF74EF3395E0FEEF25E0FF98
:103E1C00EE33FE74CE2FF58274673EF583E493F592
:103E2C0072740193F573AF74EF3395E0FEEF25E0F8
:103E3C00FFEE33FE74A42FF58274673EF583E49392
:103E4C00F570740193F571E5746403706B90001751
:103E5C00E0FFEF75F004121E50AFF0EF602E9000F3
:103E6C0016E0FFEF3395E0FEEF25E0FFEE33FE7436
:103E7C00F82FF58274673EF583E493FE740193FF8B
:103E8C00EF2571F571EE3570F570802C900016E011
:103E9C00FFEF3395E0FEEF25E0FFEE33FE74122FBB
:103EAC00F58274683EF583E493FE740193FFEF256D
:103EBC0071F571EE3570F570E576B4011090002A4D
:103ECC00E0FEA3E0FFEF4E700405778003757700EA
:103EDC00E577C394144008757700A219B39219D3EF
:103EEC00E57664809481500302419BC3E574648041
:103EFC0094864003023FC11250EAE5766404705583
:103F0C00AF74EF3395E0FE74122FF58274003EF51A
:103F1C0083E02575F0AF74EF3395E0FE74122FF546
:103F2C008274003EF583E0FFEF3395E0FED3EF950E
:103F3C0071E5706480F8EE6480984016AF73AE74CF
:103F4C00EEFD3395E0FC74122DF58274003CF58384
:103F5C00EFF0125095E5766402705AAF74EF33951A
:103F6C00E0FE74122FF58274003EF583E0FFC3EF80
:103F7C009575FFEFF0AF74EF3395E0FE74122FF5EB
:103F8C008274003EF583E0FFEF3395E0FEC3EF95BE
:103F9C0073E5726480F8EE6480985016AF71AE745D
:103FAC00EEFD3395E0FC74122DF58274003CF58324
:103FBC00EFF0125095C3E574648094865003024070
:103FCC00DD74FA2574F574E57664047072AF75EFE0
:103FDC00FD7C00AF74EF3395E0FEEF25E0FFEE3390
:103FEC00FE74242FF58274003EF583EC8DF0121FC5
:103FFC0012AF74EF3395E0FEEF25E0FFEE33FE7465
:10400C00242FF58274003EF583E0FEA3E0FFD3EF8E
:10401C009571E5706480F8EE648098401FAF74EF82
:10402C003395E0FEEF25E0FFEE33FE74242FF5828E
:10403C0074003EF583E572F0A3E573F0125199E537
:10404C0076640260030240D7AF74EF3395E0FEEF65
:10405C0025E0FFEE33FE74242FF58274003EF583C9
:10406C00C083C082E0FEA3E0FFAD757C00C3EF9D72
:10407C00FFEE9CFED082D083EEF0A3EFF0AF74EF96
:10408C003395E0FEEF25E0FFEE33FE74242FF5822E
:10409C0074003EF583E0FEA3E0FFC3EF9573E57279
:1040AC006480F8EE648098501FAF74EF3395E0FE97
:1040BC00EF25E0FFEE33FE74242FF58274003EF5FD
:1040CC0083E570F0A3E571F012519974062574F52F
:1040DC007490002AE0FEA3E0FFEF4E705CE576B42E
:1040EC000526301B230574AF74D3EF648094934082
:1040FC0003757400C21BAF74EF3395E0FE90004063
:10410C00EEF0A3EFF0125199E576640360030241DF
:10411C009B301B7B1574AF74C3EF64809480500389
:10412C00757413C21BAF74EF3395E0FE900040EE34
:10413C00F0A3EFF01251998056E576B40526301BAA
:10414C00230574AF74D3EF648094924003757400AC
:10415C00C21BAF74EF3395E0FE900040EEF0A3EF7E
:10416C00F0125199E576B40326301B231574AF7405
:10417C00C3EF648094805003757412C21BAF74EF4C
:10418C003395E0FE900040EEF0A3EFF0125199E56C
:10419C0076B40102D21BE5765406FFEF6010900056
:1041AC0040E0FEA3E0FFEF64094E7002C20F9002E4
:1041BC0007E0FEA3E0FF90002AE0FCA3E0FDED6F1A
:1041CC007002EC6E6002C20F90002AE0FEA3E0FFCA
:1041DC00900207EEF0A3EFF030A302D21A20A30A4C
:1041EC00301A07C21AA20FB3920F200F569000116B
:1041FC00E0FF8FFA90000CE0FF8FFE20800790000C
:10420C0011E02405F0900011E0FFEF3395E0FED3B0
:10421C00EF9496EE648094804005900011E4F020B9
:10422C00810790000CE02405F090000CE0FFEF33C8
:10423C0095E0FED3EF9496EE648094804005900058
:03424C000CE4F08F
:01424F00224C
:1050950012520474A012521C740212521C90001277
:1050A5007C03E01251DD12521CA3DCF6E01251DD47
:1050B500F5F0A3A3E0030354C045F012521C900081
:1050C50016E01251DD12521CC2B41251F7125204ED
:1050D50074A012521C74F012521CA3E012521CC28E
:1050E500B41251F72212520474A012521C74021207
:1050F500521C12520474A00412521C900012125237
:10510500411251E5F0A31252541252411251E5F0E9
:10511500A31252541252411251E5F0A312525412E5
:105125005241FB543F1251E5F0A312525412524121
:10513500FA541F1251E5F0EB23235403FD12524E8E
:10514500C2B41251F712520474A012521C74F01218
:10515500521C12520474A00412521C125241FB54E8
:1051650003C39D2405838007030201000302012B6D
:10517500A3F0F5F012524EC2B41251F71252047454
:10518500A012521C74F012521CE5F012521CC2B44B
:105195001251F7227AA07B807C1E90002412529433
:1051A500227AA07B8012525CED900024F07AA0A3B5
:1051B5007C1D1252C9227AA07BD07C1090006A1205
:1051C5005294227AA07BD012525CED90006AF07A5C
:0151D500A039
:1051D600A37C0F1252C92275F00A84C425F022C09E
:1051E600E0C4540F75F00AA4F5F0D0E0540F25F092
:1051F6002200D2B5000000D2B400000000221251F5
:10520600F7C2B4000000C2B500000022D2B500000B
:1052160000C2B50000227E083392B4125212DEF8A4
:1052260033D2B40000A2B450040000A2B412521249
:10523600400122C2B400001251F7227E08A2B43304
:1052460000125212DEF7C322D2B412521222C2B494
:10525600125212D2B422125204EA12521CEB125209
:105266001C125204EA0412521C125241FD12524EF2
:10527600C2B41251F722125204EA12521CEB125215
:105286001CE612521C08DCF9C2B41251F722125263
:1052960004EA12521CEB12521CE012521CA3DCF957
:1052A600C2B41251F722125204EA0412521C8003AD
:1052B600125254125241F608DCF612524EC2B41281
:1052C60051F722125204EA0412521C80031252545D
:0C52D600125241F0A3DCF612524EC2B49A
:0452E2001251F7224C
:104D9B00202020202531642E25303264202530320E
:104DAB0062753A25303262753A25303262752020B1
:104DBB0020200020202020253032642E2531642035
:104DCB0025303262753A25303262753A25303262BF
:104DDB00752020202000253033642E2531642020BF
:104DEB00253032642E25316420415A2F454C312019
:104DFB00202000253033642E2531642020253032CD
:104E0B00642E25316420415A2F454C32202020003E
:104E1B00253033642E2531642020253032642E2535
:104E2B0031642052412F444543202020002530334C
:104E3B00642E2531645720253032642E2531644E83
:104E4B00204C4F2F4C412020200025303262752002
:104E5B0020202530326275202025303262753A25AC
:104E6B00303262753A2530326275202020200025C1
:104E7B0030352E31662020253032642E25316420CA
:104E8B0020202020202025303264202000202B25BC
:104E9B003031642E2530316420202B253031642EA7
:104EAB002530316420434F52202053545020002D85
:104EBB002D2D2D2D2D2D2D2D2D2D20202020202065
:104ECB005354502000253033642E25316420202587
:104EDB003032642E25316420414E5420202531641C
:104EEB002E2531642000202020204F204520352006
:104EFB004A2046204C20202020200020202020204B
:104F0B00202020454D45202020202020202020003F
:104F1B0020416E74656E6E6120436F6E74726F6CA0
:104F2B006C65722000202020202020207620372E38
:104F3B00386120202020202020002020204A414EB4
:104F4B004645424D41524150524D41594A554E4AA8
:104F5B00554C4155475345504F43544E4F5644457E
:104F6B0043004D4F4F4E202053554E2020204341A0
:104F7B005353494F4359474E555353414749545443
:104F8B005441555255534C454F20202041515541CA
:104F9B00522E52412F444543415A2F454C32415AD0
:104FAB002F454C3100326D3A37303A32333A313388
:104FBB003A39636D36636D313047323447002053D5
:104FCB005349203130626974283732302920202030
:104FDB0020202053534931316269742831383030E5
:104FEB002920202020202053534931326269742814
:104FFB0033363030292020202020204554533235A1
:10500B0020616E6420496E6B6C2E20202020204185
:10501B00322D532D532031322062697420202020F1
:10502B00202045545332355F313062697431303250
:10503B0034202020202045545332355F31316269B2
:10504B007432303438202020202045545332355FC1
:10505B0031326269743430393620202020204D41A2
:10506B004232385F31326269743430393620202055
:10507B002020000F0C09010306171D664C030903C2
:0A508B00090309030956010102049C
:10002E00E57664016003125DD0201403020663C2FC
:10003E001430190C90002AE0FEA3E0FFEF4E601181
:10004E00900040E0FEA3E0FFEF64134E6003020158
:10005E00FB90003EE0FEA3E0FFC3EF9404EE64804D
:10006E0094804003020108AF1CAE1B126F60EF2498
:10007E0005FFEE3400FE7C007D0A121EDC9000E2CD
:10008E00EEF0A3EFF07B017A007982C003C002C0CC
:10009E00017BFF7A4D799B9000F5EBF0A3EAF0A37C
:1000AE00E9F09000E2E0FEA3E0FF7C007D64121E0A
:1000BE00DC9000F8EEF0A3EFF09000E2E0FEA3E09B
:1000CE00FF7C007D64121EDC9000FAECF0A3EDF0D4
:1000DE00900014E0FF9000FCEFF0900013E0FF9012
:1000EE0000FDEFF0900012E0FF9000FEEFF0D00167
:1000FE00D002D0031242B5020198AF1CAE1B126F94
:10010E0060EF2405FFEE3400FE7C007D0A121EDC3B
:10011E009000E2EEF0A3EFF07B017A007982C0034B
:10012E00C002C0017BFF7A4D79BE9000F5EBF0A3C3
:10013E00EAF0A3E9F09000E2E0FEA3E0FF7C007D90
:10014E000A121EDC9000F8EEF0A3EFF09000E2E051
:10015E00FEA3E0FF7C007D0A121EDC9000FAECF09C
:10016E00A3EDF0900014E0FF9000FCEFF090001370
:10017E00E0FF9000FDEFF0900012E0FF9000FEEF28
:10018E00F0D001D002D0031242B5751500D3E5159B
:10019E00648094825042AF1590003FE0FE75F003EC
:1001AE00EEA4F58285F083E5822FF582E43583F5A2
:1001BE0083E58224B0F582E583344FF583E493FF23
:1001CE00AE15EEFD3395E0FC74822DF58274003C85
:1001DE00F583EFF0051580B5C3E51B648094804070
:1001EE00030205F3900085742DF00205F390004094
:1001FE00E0FEA3E0FFEF640A4E6011900040E0FEC7
:10020E00A3E0FFEF640B4E600302029F7B017A00B6
:10021E007982C003C002C0017BFF7A4D79E1900064
:10022E00F5EBF0A3EAF0A3E9F090002CE0FEA3E0DA
:10023E00FF7C007D0A121EDC9000F8EEF0A3EFF0BA
:10024E0090002CE0FEA3E0FF7C007D0A121EDC90E5
:10025E0000FAECF0A3EDF090002EE0FEA3E0FF7CA0
:10026E00007D0A121EDC9000FCEEF0A3EFF0900071
:10027E002EE0FEA3E0FF7C007D0A121EDC9000FE45
:10028E00ECF0A3EDF0D001D002D0031242B502057E
:10029E00F3900040E0FEA3E0FFEF640C4E6011907F
:1002AE000040E0FEA3E0FFEF640D4E600302034347
:1002BE007B017A007982C003C002C0017BFF7A4DB8
:1002CE0079FE9000F5EBF0A3EAF0A3E9F090003090
:1002DE00E0FEA3E0FF7C007D0A121EDC9000F8EE2B
:1002EE00F0A3EFF0900030E0FEA3E0FF7C007D0A6B
:1002FE00121EDC9000FAECF0A3EDF0900032E0FE5E
:10030E00A3E0FF7C007D0A121EDC9000FCEEF0A341
:10031E00EFF0900032E0FEA3E0FF7C007D0A121E9B
:10032E00DC9000FEECF0A3EDF0D001D002D0031271
:10033E0042B50205F3900040E0FEA3E0FFEF640E2D
:10034E004E6011900040E0FEA3E0FFEF640F4E60A0
:10035E0003020426900036E0FEA3E0FFEF247CFFAC
:10036E00EE34FCFE90007EEEF0A3EFF090007EE007
:10037E00FEA3E0FF126F607C007D0A121EDCC00639
:10038E00C00790007EE0FEA3E0FF126F607C007D50
:10039E000A121EDC9000FEECF0A3EDF0D007D006A2
:1003AE009000FCEEF0A3EFF07B017A007982C0039F
:1003BE00C002C0017BFF7A4E791B9000F5EBF0A3D3
:1003CE00EAF0A3E9F0900034E0FEA3E0FF7C007DAC
:1003DE000A121EDC9000F8EEF0A3EFF0900034E06D
:1003EE00FEA3E0FF7C007D0A121EDC9000FAECF00A
:1003FE00A3EDF0D001D002D0031242B590007EE002
:10040E00FEA3E0FFC3EE6480948040030205F390E8
:10041E000088742DF00205F3900040E0FEA3E0FF8B
:10042E00EF64104E6011900040E0FEA3E0FFEF6419
:10043E00114E600302054D900038E0FEA3E0FFEF81
:10044E0024F8FFEE34F8FE900080EEF0A3EFF0906B
:10045E00003AE0FEA3E0FFEF247CFFEE34FCFE90BA
:10046E00007EEEF0A3EFF0900080E0FEA3E0FF121E
:10047E006F607C007D0A121EDCC006C007900080F3
:10048E00E0FEA3E0FF126F607C007D0A121EDCC04E
:10049E0004C00590007EE0FEA3E0FF126F607C00BA
:1004AE007D0A121EDCC006C00790007EE0FEA3E0AF
:1004BE00FF126F607C007D0A121EDC9000FEECF0D5
:1004CE00A3EDF0D007D0069000FCEEF0A3EFF0D035
:1004DE0005D0049000FAECF0A3EDF0D007D0069012
:1004EE0000F8EEF0A3EFF07B017A007982C003C032
:1004FE0002C0017BFF7A4E79389000F5EBF0A3EA4B
:10050E00F0A3E9F0D001D002D0031242B5900080E2
:10051E00E0FEA3E0FFC3EE64809480500690008757
:10052E007445F090007EE0FEA3E0FFC3EE6480947D
:10053E008040030205F390008D7453F00205F37BA7
:10054E00017A007982C003C002C0017BFF7A4E7926
:10055E00559000F5EBF0A3EAF0A3E9F0900015E05A
:10056E00FF9000F8EFF0900017E0FF9000F9EFF029
:10057E00900014E0FF9000FAEFF0900013E0FF906F
:10058E0000FBEFF0900012E0FF9000FCEFF0D001C6
:10059E00D002D0031242B5751500D3E515648094D0
:1005AE00825042AF15900016E0FE75F003EEA4F5F2
:1005BE008285F083E5822FF582E43583F583E5822B
:1005CE002445F582E583344FF583E493FFAE15EEB3
:1005DE00FD3395E0FC74842DF58274003CF583EFB9
:1005EE00F0051580B590002AE0FEA3E0FFC3EF945E
:1005FE0002EE648094805032900040E0FEA3E0FF53
:10060E00C3EF940AEE648094804013900040E0FEA5
:10061E00A3E0FFD3EF9411EE64809480400C900021
:10062E00947444F09000957445F07F00125DE2756D
:10063E001500D3E51564809493501AAF15EF3395DA
:10064E00E0FE74822FF58274003EF583E0FF125DAA
:10065E00A9051580DD201503020879C2159000400A
:10066E00E0FEA3E0FFC3EF940AEE64809480401591
:10067E00900040E0FEA3E0FFD3EF9411EE6480946F
:10068E00805002C2199001E4E0F8A3E0F9A3E0FA69
:10069E00A3E0FB900004E0FCA3E0FDA3E0FEA3E0DA
:1006AE00FF121A77126FD87B007A007920784112E8
:1006BE00196E7B007A007900783F12187D121BD0DC
:1006CE0090007EEEF0A3EFF09001E4E0F8A3E0F9E5
:1006DE00A3E0FAA3E0FB90007AE0FCA3E0FDA3E028
:1006EE00FEA3E0FF121A77126FD87B007A00790012
:1006FE00783F12187D121BD09000E4EEF0A3EFF0BD
:10070E007B017A00799AC003C002C0017BFF7A4E4A
:10071E00797A9000F5EBF0A3EAF0A3E9F09001E40A
:10072E00E0F8A3E0F9A3E0FAA3E0FB90000DE0FCF3
:10073E00A3E0FDA3E0FEA3E0FF121A779000F812EB
:10074E00202890007EE0FEA3E0FF7C007D0A121EB2
:10075E00DC9000FCEEF0A3EFF090007EE0FEA3E054
:10076E00FF7C007D0A121EDC9000FEECF0A3EDF083
:10077E009000E4E0FEA3E0FF900100EEF0A3EFF0A6
:10078E00D001D002D0031242B57F007E007D007CE6
:10079E0000900004E0F8A3E0F9A3E0FAA3E0FB1256
:1007AE001B1450069000A0742DF0751500D3E5159E
:1007BE00648094855042AF1590002BE0FE75F006D4
:1007CE00EEA4F58285F083E5822FF582E43583F57C
:1007DE0083E582246DF582E583344FF583E493FF40
:1007EE00AE15EEFD3395E0FC74A62DF58274003C3B
:1007FE00F583EFF0051580B590002AE0FEA3E0FF2B
:10080E00C3EF9402EE64809480400E9000AC74208E
:10081E00F09000AD7420F080217F007E007D007C82
:10082E000090007AE0F8A3E0F9A3E0FAA3E0FB124F
:10083E001B1450069000AB742DF0E5766401602B0E
:10084E007F40125DE2751500D3E5156480949350D8
:10085E001AAF15EF3395E0FE749A2FF58274003EB1
:10086E00F583E0FF125DA9051580DD201603020950
:10087E00CAC216900024E0FEA3E0FFEF249CFFEE18
:10088E0034FFFE126F60900080EEF0A3EFF0900048
:10089E0026E0FEA3E0FFEF249CFFEE34FFFE126F76
:1008AE006090007EEEF0A3EFF03010030209417B62
:1008BE00017A0079B2C003C002C0017BFF7A4E7983
:1008CE00989000F5EBF0A3EAF0A3E9F0900080E039
:1008DE00FEA3E0FF7C007D0A121EDC9000F8EEF015
:1008EE00A3EFF0900080E0FEA3E0FF7C007D0A12F3
:1008FE001EDC9000FAECF0A3EDF090007EE0FEA37B
:10090E00E0FF7C007D0A121EDC9000FCEEF0A3EFEF
:10091E00F090007EE0FEA3E0FF7C007D0A121EDC5C
:10092E009000FEECF0A3EDF0D001D002D003124205
:10093E00B580267B017A0079B2C003C002C0017B6C
:10094E00FF7A4E79BA9000F5EBF0A3EAF0A3E9F046
:10095E00D001D002D0031242B5900024E0FEA3E0F5
:10096E00FFC3EF9464EE6480948050069000B374DD
:10097E002DF0900026E0FEA3E0FFC3EF9464EE643A
:10098E0080948050069000B9742DF0E57664016075
:10099E002B7F14125DE2751500D3E51564809493D8
:1009AE00501AAF15EF3395E0FE74B22FF582740036
:1009BE003EF583E0FF125DA9051580DD20170302C9
:1009CE000BE3C217900029E0FFEF90509293FFEFD8
:1009DE003395E0FEAC66AD67121ECA8E4A8F4B9001
:1009EE0001FBE0FEA3E0FF126F607C007D0A121E89
:1009FE00DCC006C0079001FBE0FEA3E0FF126F60B3
:100A0E007C007D0A121EDC9000FEECF0A3EDF0D00F
:100A1E0007D0069000FCEEF0A3EFF07B017A007990
:100A2E00CAC003C002C0017BFF7A4E79D09000F598
:100A3E00EBF0A3EAF0A3E9F09001FDE0FEA3E0FFE6
:100A4E007C007D0A121EDC9000F8EEF0A3EFF09011
:100A5E0001FDE0FEA3E0FF7C007D0A121EDC90008B
:100A6E00FAECF0A3EDF0AE4AAF4B7C007D0A121EFD
:100A7E00DC900100EEF0A3EFF0AE4AAF4B7C007DB0
:100A8E000A121EDC900102ECF0A3EDF0D001D002B0
:100A9E00D0031242B59001FBE0FEA3E0FFC3EE646B
:100AAE0080948050069000D0742DF0A21CB3921C3E
:100ABE00E508540CFFEFB40808201C059000DAE49A
:100ACE00F0E508540CFFEFB40409201C069000DA80
:100ADE007401F0E508540CFFEFB40C09300F0690CA
:100AEE0000DA742AF0E5085403FFEFB40209301C53
:100AFE00069000D97402F0E5085403FFEFB4010923
:100B0E00301C069000D97403F0E5085403FFEFB4CF
:100B1E000309300F069000D9742AF0900040E0FED1
:100B2E00A3E0FFEF64124E6003020BB8751500D3FD
:100B3E00E515648094935042AF1590003DE0FE752C
:100B4E00F014EEA4F58285F083E5822FF582E4356C
:100B5E0083F583E58224C9F582E583344FF583E47A
:100B6E0093FFAE15EEFD3395E0FC74CA2DF582743D
:100B7E00003CF583EFF0051580B5AE4AAF4B7C0017
:100B8E007D0A121EDCEF2430FF9000DBEFF09000A8
:100B9E00DC742EF0AE4AAF4B7C007D0A121EDCAF29
:100BAE0005EF2430FF9000DDEFF07F54125DE2750B
:100BBE001500D3E51564809493501AAF15EF339555
:100BCE00E0FE74CA2FF58274003EF583E0FF125DDD
:100BDE00A9051580DDE576B40114900041E0FFEF24
:100BEE0090507E93FF125DE2125DC7125DD93018F0
:100BFE0003020D467B017A007982C003C002C00158
:100C0E007BFF7A4E79F19000F5EBF0A3EAF0A3E9C1
:100C1E00F0D001D002D0031242B57B017A00799A4E
:100C2E00C003C002C0017BFF7A4F79069000F5EB3E
:100C3E00F0A3EAF0A3E9F0D001D002D0031242B53E
:100C4E007B017A0079B2C003C002C0017BFF7A4FEC
:100C5E00791B9000F5EBF0A3EAF0A3E9F0D001D0F8
:100C6E0002D0031242B57B017A0079CAC003C002DA
:100C7E00C0017BFF7A4F79309000F5EBF0A3EAF0DC
:100C8E00A3E9F0D001D002D0031242B57F00125D6D
:100C9E00E2751500D3E51564809493501AAF15EFE5
:100CAE003395E0FE74822FF58274003EF583E0FFEB
:100CBE00125DA9051580DD7F40125DE2751500D32A
:100CCE00E51564809493501AAF15EF3395E0FE74DA
:100CDE009A2FF58274003EF583E0FF125DA905158B
:100CEE0080DD7F14125DE2751500D3E515648094E6
:100CFE0093501AAF15EF3395E0FE74B22FF5827450
:100D0E00003EF583E0FF125DA9051580DD7F5412CC
:100D1E005DE2751500D3E51564809493501AAF15F6
:100D2E00EF3395E0FE74CA2FF58274003EF583E032
:090D3E00FF125DA9051580DD22FC
:106E2D00015100014F00015000014900C10FC10C7B
:0A6E3D00C10BC10EC110C10DC1113F
:106F7200752400D3E524648094A75004052480F38B
:016F820022EC
:106F8300752500D3E525648094935004052580F38B
:016F930022DB
:106F9400752600D3E5266480949E5004052680F36C
:016FA40022CA
:106FA500752700D3E5276480949E5004052780F358
:016FB50022B9
:106FB600752800C3E5286480949E5004052880F354
:016FC60022A8
:106FC700752900C3E529648094815004052980F35D
:016FD7002297
:10626D00C292C296126F72126F72C290126F7275D5
:10627D002F1F752E00E52ED394075011E52FC31354
:10628D00F52FA2D79290126F72052E80E8D2901240
:10629D006F72D292752A03752BE8752F003091100D
:1062AD00E52B152B7002152A14FFAE2AEF4E70ED5B
:1062BD00126F83752E00E52ED394075013126F7253
:1062CD00E52FC313F52F309103432F80052E80E664
:1062DD00126F72AF2F7E00EF752D00F52C752A030E
:1062ED00752BE8752F00309110E52B152B700215CD
:1062FD002A14FFAE2AEF4E70ED126F83752E00E556
:10630D002ED394075013126F72E52FC313F52F3050
:10631D009103432F80052E80E6126F72AF2F7E0002
:10632D00EF252DF52DEE352CF52CC3E52C64809441
:10633D00805006752C00752D00D3E52D940FE52C9E
:10634D006480948E4006752C0E752D0F20B20DC3F2
:10635D00740F952DF52D740E952CF52CAE2CAF2DAF
:01636D00220D
:10645E00C294126F7275351F753400E534D39407EC
:10646E005011E535C313F535A2D79294126F72050C
:10647E003480E8D294126F72D2967530037531E87B
:10648E00753500309510E53115317002153014FF59
:10649E00AE30EF4E70ED126F83753400E534D39449
:1064AE00075013126F72E535C313F535309503435C
:1064BE003580053480E6126F72AF357E00EF75338E
:1064CE0000F5327530037531E8753500309510E5FD
:1064DE003115317002153014FFAE30EF4E70ED12E3
:1064EE006F83753400E534D394075013126F72E541
:1064FE0035C313F535309503433580053480E612E8
:10650E006F72AF357E00EF2533F533EE3532F5324F
:10651E00C3E532648094805006753200753300D323
:10652E00E533940FE5326480948E400675320E7515
:06653E00330FAE32AF3353
:016544002234
:10000E0012626D8E4D8F4E12645E8E478F487566EE
:05001E000075670122DE
:10697D00D290D294D291D295756C00756D007568D8
:10698D0000756900753600D3E536648094895049E9
:10699D00126F94C290C294126F94C3E536648094C2
:1069AD00895004D290D294E56D256DF56DE56C3569
:1069BD006CF56CE5692569F569E5683568F568205C
:1069CD009108056DE56D7002056C2095080569E56A
:1069DD006970020568053680AEC290C29475660076
:1069ED00756705AE6CAF6D7C007D05121ECA8E4DB0
:1069FD008F4E20B20DC3740B954EF54E740E954D02
:106A0D00F54DAE68AF697C007D05121ECA8E478FAD
:016A1D004830
:016A1E002255
:106B5900D290D294D291D295756C00756D007568FA
:106B690000756900753700D3E5376480948A504908
:106B7900126F94C290C294126F94C3E537648094E3
:106B89008A5004D290D294E56D256DF56DE56C358A
:106B99006CF56CE5692569F569E5683568F568207E
:106BA9009108056DE56D7002056C2095080569E58C
:106BB9006970020568053780AEC290C29475660097
:106BC900756702E56D25E0F54EE56C33F54D20B2AC
:106BD9000DC3740E954EF54E740E954DF54DE56940
:096BE90025E0F548E56833F547A5
:016BF2002280
:106D1900D290D294D291D295756C00756D00756838
:106D290000756900753800D3E5386480948B504943
:106D3900126F94C290C294126F94C3E53864809420
:106D49008B5004D290D294E56D256DF56DE56C35C7
:106D59006CF56CE5692569F569E5683568F56820BC
:106D69009108056DE56D7002056C2095080569E5CA
:106D79006970020568053880AEC290C294756600D4
:106D8900756701856C4D856D4E20B20DC3740F95E5
:0F6D99004EF54E740E954DF54D8568478569484A
:016DA80022C8
:105E2700D292D291756C00756D00126FA57539000D
:105E3700D3E5396480948F5025D290126FA5C29014
:105E4700126FA5E56D256DF56DE56C356CF56C206C
:105E57009108056DE56D7002056C053980D2C29019
:105E6700C292E56DAE6C7806CEC313CE13D8F9F5A2
:105E77006D8E6CAC6CAD6DE4121B977B007A00796C
:105E870034784412196E7B007A0079807844121AAC
:105E970077121BD07C007D05121ECA8E4D8F4E20B7
:105EA700B20DC3740B954EF54E740E954DF54D120C
:105EB7006FA5756600756705D296D29575680075EA
:105EC7006900126FA5753900D3E5396480948F5046
:105ED70025D294126FA5C294126FA5E5692569F5BD
:105EE70069E5683568F5682095080569E569700210
:105EF7000568053980D2C294C296E569AE6878060E
:105F0700CEC313CE13D8F9F5698E68AC68AD69E4D2
:105F1700121B977B007A007934784412196E7B0044
:105F27007A0079807844121A77121BD07C007D059D
:075F3700121ECA8E478F48BD
:015F3E002240
:105F3F00D292D291756C00756D00126FA5753A00F3
:105F4F00D3E53A6480948F5025D290126FA5C290FA
:105F5F00126FA5E56D256DF56DE56C356CF56C2053
:105F6F009108056DE56D7002056C053A80D2C290FF
:105F7F00C292E56DAE6C7805CEC313CE13D8F9F58A
:105F8F006D8E6CAC6CAD6DE4121B977B007A007953
:105F9F00E1784412196E7B007A0079007845121A65
:105FAF0077121BD0EF25E0F54EEE33F54D20B20DF5
:105FBF00C3740E954EF54E740E954DF54D126FA59B
:105FCF00756600756702D296D2957568007569007F
:105FDF00126FA5753A00D3E53A6480948F5025D29D
:105FEF0094126FA5C294126FA5E5692569F569E54D
:105FFF00683568F5682095080569E56970020568D8
:10600F00053A80D2C294C296E569AE687805CEC3D0
:10601F0013CE13D8F9F5698E68AC68AD69E4121B1D
:10602F00977B007A0079E1784412196E7B007A0031
:10603F0079007845121A77121BD0EF25E0F548EE5C
:03604F0033F547DF
:01605200222B
:10616100D292D291756C00756D00126FA5753B00CE
:10617100D3E53B6480948F5025D290126FA5C290D5
:10618100126FA5E56D256DF56DE56C356CF56C202F
:106191009108056DE56D7002056C053B80D2C290DA
:1061A100C292E56CC4F854F0C868F56CE56DC4544E
:1061B1000F48F56DAC6CAD6DE4121B977B007A0056
:1061C1007961784512196E7B007A007980784512E1
:1061D1001A77121BD08E4D8F4E20B20DC3740F95BE
:1061E1004EF54E740E954DF54D126FA57566007501
:1061F1006701D296D295756800756900126FA57511
:106201003B00D3E53B6480948F5025D294126FA557
:10621100C294126FA5E5692569F569E5683568F5E8
:10622100682095080569E56970020568053B80D21B
:10623100C294C296E568C4F854F0C868F568E56987
:10624100C4540F48F569AC68AD69E4121B977B0033
:106251007A007961784512196E7B007A007980782D
:0B62610045121A77121BD08E478F48A1
:01626C00220F
:10605300D292D291756C00756D00126FA5753C00DC
:10606300D3E53C6480948F5025D290126FA5C290E3
:10607300126FA5E56D256DF56DE56C356CF56C203E
:106083009108056DE56D7002056C053C80D2C290E8
:10609300C292E56CC4F854F0C868F56CE56DC4545D
:1060A3000F48F56DAC6CAD6DE4121B977B007A0065
:1060B3007961784512196E7B007A007980784512F0
:1060C3001A77121BD08E4D8F4E20B20DC3740F95CD
:1060D3004EF54E740E954DF54D126FA57566007510
:1060E3006701D295756800756900126FC7753C002A
:1060F300D3E53C6480948C5032C294126FC7D2941F
:10610300D294D294D294D294D294D294D294D2945C
:10611300E5692569F569E5683568F5682095080539
:1061230069E56970020568053C80C5D294E568C3DA
:1061330013F568E56913F569AC68AD69E4121B975B
:106143007B007A007961784512196E7B007A0079B9
:0D615300807845121A77121BD08E478F48B6
:01616000221C
:1058BC00D292D291756C00756D00126FB6753D0069
:1058CC00D3E53D6480948F5025D290126FB6C29070
:1058DC00126FB6E56D256DF56DE56C356CF56C20CC
:1058EC009108056DE56D7002056C053D80D2C29086
:1058FC00C292E56CC4F854F0C868F56CE56DC454FC
:10590C000F48F56DD3E56D9559E56C9558401885A4
:10591C006C62856D63856C58856D59E56D24FFF55A
:10592C0057E56C34FFF556C3E56D9557E56C955608
:10593C00501EE56D2401F563E56C3400F562856C51
:10594C0056856D57E56D2401F559E56C3400F55815
:10595C00AC62AD63EC121B977B007A0079617845E1
:10596C0012196E7B007A0079807845121A77121B17
:10597C00D08E4D8F4E20B20DC3740F954EF54E74D4
:10598C000E954DF54D126FA5756600756701D29693
:10599C00D295756800756900126FB6753D00D3E538
:1059AC003D6480948F5025D294126FB6C294126FBE
:1059BC00B6E5692569F569E5683568F568209508E7
:1059CC000569E56970020568053D80D2C294C296EE
:1059DC00E568C4F854F0C868F568E569C4540F4824
:1059EC00F569D3E5699555E5689554401885685E69
:1059FC0085695F856854856955E56924FFF553E52C
:105A0C006834FFF552C3E5699553E5689552501E0D
:105A1C00E5692401F55FE5683400F55E856852851B
:105A2C006953E5692401F555E5683400F554AC5E1D
:105A3C00AD5FEC121B977B007A00796178451219E7
:105A4C006E7B007A0079807845121A77121BD08E03
:035A5C00478F4829
:015A5F002224
:1038BC00E54C64326003300D60C3E56F954EF561E5
:1038CC00E56E954DF560C374089548FF74079547F0
:1038DC00FE126F60EF247CFFEE34FCFEC3E56B9FA1
:1038EC00F55BE56A9EF55AC3E5489408E5476480A4
:1038FC009487500BC3E4955BF55BE4955AF55AC27B
:10390C0010C20E90006AE560F0A3E561F090006CC7
:10391C00E55AF0A3E55BF0C20D20101B20B3033079
:10392C000E03301112D210D20E90006EE4F0A3747C
:10393C0001F01251BBC21130101D20B303300E0325
:10394C00301114C210D20E1251A690006EE4F0A3E6
:10395C00E4F01251BBC21120B304054C8005754C28
:10396C0000C20E301074E561254EF54EE560354D04
:10397C00F54DD3E54E940FE54D6480948E400C7458
:10398C00F0254EF54E74F1354DF54DC3E54D648083
:10399C009480500C7410254EF54E740E354DF54D2B
:1039AC00E55B2548F548E55A3547F547D3E5489496
:1039BC000FE5476480948E400C74F02548F54874EC
:1039CC00F13547F547C3E54764809480500C74107B
:1039DC002548F548740E3547F547C374089548FFDC
:1039EC0074079547FE126F60EF247CF548EE34FCAB
:1039FC00F5479001FDE54DF0A3E54EF09001FBE598
:103A0C0047F0A3E548F0E56F24F8F55DE56E34F872
:103A1C00F55CE54E24F8F565E54D34F8F564C3E541
:103A2C005C64809480500C7410255DF55D740E35CB
:103A3C005CF55CC3E56464809480500C741025655F
:103A4C00F565740E3564F56430105A90003AE0FE5A
:103A5C00A3E0FFC3EF9484EE64809483400FC3E52E
:103A6C006F954EF53FE56E954DF53E800DC3E55DCA
:103A7C009565F53FE55C9564F53ED3E56B9400E503
:103A8C006A648094804010C3E56B9548F541E56A03
:103A9C009547F540023B59C3E49548F541E49547F9
:103AAC00F540023B5990003AE0FEA3E0FFC3EF94CF
:103ABC0084EE648094834025900024E0FEA3E0FF14
:103ACC00E56F2FFFE56E3EFEEF249CFFEE34FFFE0C
:103ADC00C3EF954EF53FEE954DF53E8023900024B7
:103AEC00E0FEA3E0FFE55D2FFFE55C3EFEEF249CCE
:103AFC00FFEE34FFFEC3EF9565F53FEE9564F53EA2
:103B0C00D3E56B9400E56A64809480402590002690
:103B1C00E0FEA3E0FFE56B2FFFE56A3EFEEF249C81
:103B2C00FFEE34FFFEC3EF9548F541EE9547F540A7
:103B3C00801B900026E0FEA3E0FFEF249CFFEE34F8
:103B4C00FFFEC3EF9548F541EE9547F54075080F1C
:103B5C00200F03023D91AE4AAF4B7C007D02121E3A
:103B6C00DCD3E53F9FEE6480F8E53E64809840240A
:103B7C00E54620E5067551007550000551AF51EF33
:103B8C00D394504003755150E551C3940A4050539F
:103B9C00080E804BAE4AAF4B7C007D02121EDCC37C
:103BAC00E49FFFE49EFEC3E53F9FEE6480F8E53E94
:103BBC006480985024E54620E40675510075500049
:103BCC000551AF51EFD394504003755150E551C39B
:103BDC00940A400B53080D8006755100755000AEC9
:103BEC004AAF4B7C007D02121EDCD3E5419FEE6494
:103BFC0080F8E5406480984024E54620E706754F40
:103C0C0000754900054FAF4FEFD394504003754FEB
:103C1C0050E54FC3940A405D53080B8058AE4AAF31
:103C2C004B7C007D02121EDCC3E49FFFE49EFEC3AE
:103C3C00E5419FEE6480F8E5406480985031D3E50F
:103C4C00489400E547648094804024E54620E606CD
:103C5C00754F00754900054FAF4FEFD3945040039B
:103C6C00754F50E54FC3940A400B530807800675F7
:103C7C004F00754900AF3FAE3E126F608E428F43CE
:103C8C00C374289543FFE49542FEEF7802C333CE0C
:103C9C0033CED8F9FFAD507C00C3EF9DF545EE9CBB
:103CAC00F544C3E544648094805006754400754522
:103CBC0000E551C39450501DAF517E007C007D7FB8
:103CCC00121ECA7C007D50121EDCEF2480FFEF64B4
:103CDC00FFF5FA8027C3E5439428E542648094807D
:103CEC005017E550C394A050100550C3E5446480B0
:103CFC00948040088545FA800375FA00AF41AE40C8
:103D0C00126F608E428F43C374289543FFE4954233
:103D1C00FEEF7802C333CE33CED8F9FFAD497C0029
:103D2C00C3EF9DF545EE9CF544C3E5446480948057
:103D3C005006754400754500E54FC39450501DAFB7
:103D4C004F7E007C007D7F121ECA7C007D50121EAF
:103D5C00DCEF2480FFEF64FFF5FE8035C3E5439470
:103D6C0028E542648094805017E549C394A0501014
:103D7C000549C3E5446480948040168545FE801156
:103D8C0075FE00800C755100755000754F0075491B
:0F3D9C0000E508C454F0FFEF240FF5468546A05C
:013DAB0022F5
:106EE1004310000043D8000044A2000045110000F7
:106EF1004554800045B400004622000046BD000014
:106F010000C700C70002000A0E0F03840E0F03849E
:106F1100000100010000000000000000000000006E
:106E4700011400011663011200011700011A00C1A5
:036E570013C192D2
:0300030002660D85
:10660D00C0E0C083C08263A201C083C082C0D075C8
:10661D00D000C006C00720124F20134CD2B330B3A8
:10662D00020512051AAF1AC3EF64809488401CAF9F
:10663D0017EF3395E0FE74422FF58274003EF5831B
:10664D00E512F07512000517751A00E5122512F501
:10665D0012C3E51764809484404F751700D21390D0
:10666D00004AE0FF8F12804120123E30133BE512AD
:10667D002512F512A2D792B3051AAF1AC3EF648093
:10668D009488401A0517AF17EF3395E0FE744A2F23
:10669D00F58274003EF583E0FF8F12751A00C3E595
:1066AD0017648094A04002D212D007D006D0D0D06B
:0D66BD0082D08363A201D082D083D0E0326E
:10550E0090004AE56EF0A3E56FF0E56B2484FFE5AD
:10551E006A3403FE90004CEEF0A3EFF09001FDE034
:10552E00FEA3E0FF90004EEEF0A3EFF09001FBE043
:10553E00FEA3E0FFEF2484FFEE3403FE900050EE56
:10554E00F0A3EFF0E50B2484FFE50A3403FE900090
:10555E0052EEF0A3EFF0900024E0FEA3E0FF9000E7
:10556E0054EEF0A3EFF0900026E0FEA3E0FF9000D3
:10557E0056EEF0A3EFF090002AE0FEA3E0FF9000BD
:10558E0058EEF0A3EFF090005AE54AF0A3E54BF089
:10559E00300F0B90005CE4F0A37401F080089000D3
:1055AE005CE4F0A3E4F0900017E0FFEF3395E0FE2B
:1055BE0090005EEEF0A3EFF0900016E0FFEF339553
:1055CE00E0FE900060EEF0A3EFF0900015E0FFEF2C
:1055DE003395E0FE900062EEF0A3EFF0900014E041
:1055EE00FFEF3395E0FE900064EEF0A3EFF0900035
:1055FE0013E0FFEF3395E0FE900066EEF0A3EFF0C0
:10560E00900043E0F516900042E4F0A37463F0C3FB
:10561E00E5166480948840030256FFC3E516648045
:10562E00948050030256FF900044E0F518A3E0F575
:10563E0019AF16EF3395E0FEEF25E0FFEE33FE7463
:10564E00012FF582746F3EF583E493FE740193FF90
:10565E00D3E5199FEE6480F8E5186480984021AF79
:10566E0016EF3395E0FEEF25E0FFEE33FE74012FCB
:10567E00F582746F3EF583E493F518740193F51972
:10568E00AF16EF3395E0FEEF25E0FFEE33FE74111B
:10569E002FF582746F3EF583E493FE740193FFC37E
:1056AE00E5199FEE6480F8E5186480985021AF16D6
:1056BE00EF3395E0FEEF25E0FFEE33FE74112FF58C
:1056CE0082746F3EF583E493F518740193F519AF68
:1056DE0016EF3395E0FEEF25E0FFEE33FE74242F38
:1056EE00F58274003EF583E518F0A3E519F012512A
:0C56FE0099E516B40805A20FB3920F2224
:03002B0002654526
:10654500C0E0C0F0C083C08263A201C083C082C026
:10655500D075D000C000C001C002C003C004C00592
:10656500C006C00775A61E75A6E11509AF09EF702F
:106575007330187075090443800353907790003C7D
:10658500E0FEA3E0FFEF8EF01220AB65B8000065DA
:10659500BD000165C2000265C7000365CC00046546
:1065A500D1000565D6000665DB000765E00008003B
:1065B5000065E312697D8026126B598021126D19E1
:1065C500801C126053801712000E8012125E278005
:1065D5000D125F3F800812616180031258BC439021
:1065E500881238BCC2CFD007D006D005D004D0035E
:1065F500D002D001D000D0D0D082D08363A201D008
:0866050082D083D0F0D0E03216
:03002300026DA9C2
:106DA900C0E0C0F0C083C08263A201C083C082C0BA
:106DB900D075D000C000C001C002C003C004C00526
:106DC900C006C007C2AC30981AC298E599B43F030F
:106DD9001252E6E599B4210B12570AD214D215D2F0
:106DE90016D217C299D2ACD007D006D005D004D09C
:106DF90003D002D001D000D0D0D082D08363A201C9
:096E0900D082D083D0F0D0E03239
:03000B000266CAC0
:1066CA00C0E0C0F0C083C08263A201C083C082C0A0
:1066DA00D075D000C000C001C002C003C004C0050C
:1066EA00C006C007758A00758C4C75A61E75A6E192
:1066FA00E513B42802C2960514AF14C3EF6480945C
:10670A008A4016301213751400751700751A00C2E4
:10671A0013C21275120012550EE51375F007121EF8
:10672A0050AFF0EF701B123DAC301804D214D217E0
:10673A00E5766007301804D215D21612002E1250D0
:10674A00EA1513AF13EF700C75134ED218301804F4
:10675A00D215D216D007D006D005D004D003D00265
:10676A00D001D000D0D0D082D08363A201D082D011
:06677A0083D0F0D0E032F4
:10224500758FFF758921758DFF438780759850D2ED
:102255008CD28ED2CA75CB4C75CA0043B71143B820
:1022650021D28875D90243D84075DA4275DE42C25B
:10227500187513467509017F02125D71125DBE75F1
:102285007700900042E4F0A37463F020A003126B82
:10229500F375A8B275A7071251A61251C89000117F
:1022A500E4F090000CE4F0C20F90006EE0FEA3E0B5
:1022B500FFEF4E6004D2108002C21090006AE0F574
:1022C50060A3E0F56190006CE0F55AA3E0F55BE5ED
:1022D5007670FC900038E0FCA3E0FDEC121B977BC8
:1022E500007A0079207841121A777B007A007934D8
:1022F50078C312187D9001E4E0F8A3E0F9A3E0FAB1
:10230500A3E0FB12196E90002012202890003AE0FD
:10231500FCA3E0FDEC121B977B007A007920784145
:10232500121A777B007A0079B478C212187D900171
:10233500E4E0F8A3E0F9A3E0FAA3E0FB12196E903C
:10234500001C122028900013E0FCEC121B9C7B0063
:102355007A0079B47844121A77C004C005C006C063
:1023650007900014E0FCEC121B9C7B007A0079C0FE
:102375007841121A77A804A905AA06AB07D007D099
:1023850006D005D00412187DC004C005C006C007DC
:10239500900012E0FCEC121B9C7B007AC079A878B7
:1023A50047121A77A804A905AA06AB07D007D006D5
:1023B500D005D00412187D900046122028900016F2
:1023C500E0FFEF3395E0FEFDFCEF2409FFEE34005E
:1023D500FEED3400FDEC3400FC7B0C7A00790078CE
:1023E50000126E5BA804A905AA06AB07900017E0CA
:1023F500FFEF3395E0FEFDFCEF24D0FFEE3407FE42
:10240500ED3400FDEC3400FCEB2FFFEA3EFEE93D28
:10241500FDE83CFC7B077A0079007800121F287BD9
:10242500047A0079007800126E5BC004C005C0060E
:10243500C007900017E0FFEF3395E0FEFDFC7B6FD2
:102445007A0179007800121F28D003D002D001D07C
:1024550000C3EF9BFFEE9AFEED99FDEC98FCC004DE
:10246500C005C006C007900016E0FFEF3395E0FEFB
:10247500FDFC7B137A0179007800121F287B097A0D
:102485000079007800126E5BA804A905AA06AB07BF
:10249500D007D006D005D004EB2FFBEA3EFAE93D84
:1024A500F9E83CF8900015E0FFEF3395E0FEFDFC00
:1024B500EB2FFFEA3EFEE93DFDE83CFCEF247AF513
:1024C50011EE34E0F510ED3400F50FEC3400F50EA7
:1024D50090002AE0FEA3E0FFEF64014E70487B0107
:1024E5007A007908C003C002C0017B017A00797ABD
:1024F5009001ADEBF0A3EAF0A3E9F0AF11AE10AD9A
:102505000FAC0E9001B0122028900046E0FCA3E02D
:10251500FDA3E0FEA3E0FF9001B4122028D001D076
:1025250002D0031246D390002AE0FEA3E0FFEF4E4F
:1025350060030227C97B017A007908C003C002C085
:10254500017B017A00797A900125EBF0A3EAF0A3EB
:10255500E9F0AF11AE10AD0FAC0E90012812202896
:10256500900046E0FCA3E0FDA3E0FEA3E0FF9001A0
:102575002C122028D001D002D003122B9EAF11AE11
:1025850010AD0FAC0EC004C005C006C007900046D4
:10259500E0FCA3E0FDA3E0FEA3E0FF9001601220B4
:1025A50028D007D006D005D004120D47A804A905E8
:1025B500AA06AB077F007E3E7DC67C481218797B54
:1025C500007A00797A7844121A77A804A905AA0630
:1025D500AB077F007EC07D3C7C45121879C004C0E6
:1025E50005C006C00790001CE0FCA3E0FDA3E0FECB
:1025F500A3E0FF125AA8A804A905AA06AB07D007AD
:10260500D006D005D00412196EC004C005C006C09E
:1026150007900018E0FCA3E0FDA3E0FEA3E0FF1295
:102625005ABEA804A905AA06AB07D007D006D0054F
:10263500D00412196EC004C005C006C00790007A08
:10264500E0FCA3E0FDA3E0FEA3E0FF125AA8A80466
:10265500A905AA06AB07D007D006D005D0041219E4
:102665006EC004C005C006C007AF11AE10AD0FACFB
:102675000EC004C005C006C0077FAB7EAA7D0A7CDC
:10268500BF900046E0F8A3E0F9A3E0FAA3E0FB124F
:10269500187D900160122028D007D006D005D004FF
:1026A500120D47C004C005C006C007AF11AE10AD7E
:1026B5000FAC0EC004C005C006C0077F007E007DBC
:1026C500207CBF900046E0F8A3E0F9A3E0FAA3E080
:1026D500FB12187D900160122028D007D006D00586
:1026E500D004120D47D003D002D001D000121879C2
:1026F5007B337A337993783F121A77A804A905AA10
:1027050006AB07D007D006D005D00412187D121BE2
:10271500D08E0C8F0D90003EE0FEA3E0FFC3EF943A
:1027250004EE64809480504FAC0CAD0DEC121B97F9
:10273500C004C005C006C00790003EE0FEA3E0FF50
:10274500EF7802C333CE33CED8F9FF74E12FF5828B
:10275500746E3EF583121FF8D007D006D005D0045D
:1027650012196E7B007A00797A7844121A77121B57
:10277500D08E1B8F1C804DAC0CAD0DEC121B97C081
:1027850004C005C006C00790003EE0FEA3E0FFEFD1
:102795007802C333CE33CED8F9FF74E12FF58274B6
:1027A5006E3EF583121FF8D007D006D005D004126F
:1027B500196E7B007A40791C7846121A77121BD065
:1027C5008E1B8F1C90002AE0FEA3E0FFEF64024EF3
:1027D500701490007A1220343F82D0E590000812E0
:1027E500203440C39DB290002AE0FEA3E0FFEF64D1
:1027F500034E701490007A1220343F3566CF900056
:102805000812203440A73B6490002AE0FEA3E0FFB5
:10281500EF64044E701490007A122034BF018FC506
:1028250090000812203440953F7D90002AE0FEA3D9
:10283500E0FFEF64054E701490007A1220343EC418
:102845004D019000081220343FB9168790002AE008
:10285500FEA3E0FFEF64064E701490007A12203458
:102865003F32B6AE900008122034401F2B02900074
:102875002AE0FEA3E0FFEF64074E701490007A1281
:1028850020340000000090000812203440BC7AE19A
:1028950090002AE0FEA3E0FFEF64084E7067900009
:1028A50034E0FCA3E0FDEC121B977B007A00792055
:1028B5007841121A779001E4E0F8A3E0F9A3E0FA71
:1028C500A3E0FB12196E900008122028900036E054
:1028D500FCA3E0FDEC121B977B007A007920784180
:1028E500121A777B007A0079B478C212187D9001AC
:1028F500E4E0F8A3E0F9A3E0FAA3E0FB12196E9077
:10290500007A12202890002AE0FEA3E0FFC3EF948E
:1029150009EE648094804003022A1D900046E0FC85
:10292500A3E0FDA3E0FEA3E0FFC004C005C006C010
:1029350007AF11AE10AD0FAC0E9001D0122028D00C
:1029450007D006D005D004124A9B90018A12202890
:102955007B017A00790DC003C002C0017B017A00BA
:102965007900900187EBF0A3EAF0A3E9F090000865
:10297500E0FCA3E0FDA3E0FEA3E0FF90018E1220A2
:102985002890007AE0FCA3E0FDA3E0FEA3E0FF9021
:102995000192122028D001D002D0031233A5900055
:1029A5002AE0FEA3E0FFEF4E705A900000E0FCA382
:1029B500E0FDA3E0FEA3E0FF125AA87B007A507960
:1029C500C7784512196EC004C005C006C00790003F
:1029D500EA12203448B98C00D007D006D005D004BF
:1029E500126ABCA804A905AA06AB07900000E0FC82
:1029F500A3E0FDA3E0FEA3E0FF1218799000041206
:102A050020288014900000E0FCA3E0FDA3E0FEA3D5
:102A1500E0FF90000412202890002AE0FEA3E0FFCA
:102A2500EF64094E705C900030E0FCA3E0FDEC1211
:102A35001B977B007A0079207841121A779001E480
:102A4500E0F8A3E0F9A3E0FAA3E0FB12196E900009
:102A55000D122028900032E0FCA3E0FDEC121B973C
:102A65007B007A0079207841121A779001E4E0F82A
:102A7500A3E0F9A3E0FAA3E0FB12196E900004129B
:102A8500202890002AE0FEA3E0FFEF640A4E705C68
:102A950090002CE0FCA3E0FDEC121B977B007A0074
:102AA50079207841121A779001E4E0F8A3E0F9A3C0
:102AB500E0FAA3E0FB12196E90000D122028900099
:102AC5002EE0FCA3E0FDEC121B977B007A00792039
:102AD5007841121A779001E4E0F8A3E0F9A3E0FA4F
:102AE500A3E0FB12196E9000041220289001E4E087
:102AF500F8A3E0F9A3E0FAA3E0FB90000DE0FCA346
:102B0500E0FDA3E0FEA3E0FF121A777BCD7ACC7936
:102B15004C783D12187D7B007A0079207841121996
:102B25006E121BD08E6E8F6F9001E4E0F8A3E0F972
:102B3500A3E0FAA3E0FB900004E0FCA3E0FDA3E022
:102B4500FEA3E0FF121A777BCD7ACC794C783D1243
:102B5500187D7B007A007920784112196E121BD0FE
:102B65008E6A8F6B7F007E007D207C4190007AE02D
:102B7500F8A3E0F9A3E0FAA3E0FB12196E9001E4D3
:102B8500E0F8A3E0F9A3E0FAA3E0FB121A77121B21
:092B9500D08E0A8F0B0222D4221B
:105D0A00EFC0E0C283740F125D3F7430125D4974B4
:105D1A0005125D3F7430125D497401125D3F7430A3
:105D2A00125D497401125D3FD0E0146002740844A8
:105D3A0020125D57227D000000DDFCD5E0F72254D9
:105D4A00F053800F4280C282D283C28322C28280F1
:105D5A0002D282C0E0125D65D0E0C454F053800FD5
:105D6A004280D283C28322125D0A125DA374061294
:105D7A005D57125DA3740E125D57125DA374011272
:105D8A005D57125DA37440125D57125DF0125DA358
:105D9A007480125D57125DD022740A125D3F22EFA1
:105DAA00C0E0125DA3D0E0125D5B22125DA3740213
:105DBA00125D5722125DA37401125D5722125DA370
:105DCA00740E125D5722125DA3740C125D572212D3
:105DDA005DA3740F125D5722EFC0E0125DA3D0E0FD
:105DEA004480125D5722905DFF7E28E493FF125D86
:105DFA00A9A3DEF7220004040E0E1F1F00001F1FB6
:105E0A000E0E04040000101C1F1C100000000107E5
:0D5E1A001F070100000E11171917110E00CF
:106F48007A107B00EE6BFB8BF053F080ABF033EFE5
:086F580033FFEE33FEDAEE22F6
:106C8800900209EEF0A3EFF0900209E0FEA3E0FF06
:106C98007C037DE8121EDCEF2430F5993099FDC2A3
:106CA80099900209E0FEA3E0FF7C037DE8121EDC58
:106CB8007E007F64CFCDCFCECCCE121EDCEF243049
:106CC800F5993099FDC299900209E0FEA3E0FF7C96
:106CD800007D64121EDC7E007F0ACFCDCFCECCCEE5
:106CE800121EDCEF2430F5993099FDC29990020903
:106CF800E0FEA3E0FF7C007D0A121EDCAF05EF2456
:106D080030F5993099FDC2997599003099FDC2996D
:016D18002258
:1052E6009001FF122034000186A020983E9001FF15
:1052F600E0FCA3E0FDA3E0FEA3E0FFEC4D4E4F6013
:105306002A9001FFE0FCA3E0FDA3E0FEA3E0FF7B03
:10531600FF7AFF79FF78FFEF2BFFEE3AFEED39FDBE
:10532600EC38FC9001FF12202880BFC298AF99EF9D
:10533600122085538B6153976253A36353AB645317
:10534600B76553C36653CF6753DB6853E76953F3B7
:105356006A53FF6B540B6C54176D54236E54316FA4
:10536600543D705451715459725467735475745442
:10537600BA7554C87654D67754E47854F279550001
:105386007A0000550D900024E0FEA3E0FF126C8821
:1053960022900026E0FEA3E0FF126C8822AF4BAEFF
:1053A6004A126C882290002AE0FEA3E0FF126C8865
:1053B6002290002CE0FEA3E0FF126C882290002EC3
:1053C600E0FEA3E0FF126C8822900030E0FEA3E02E
:1053D600FF126C8822900032E0FEA3E0FF126C8878
:1053E60022900034E0FEA3E0FF126C882290003683
:1053F600E0FEA3E0FF126C8822900038E0FEA3E0F6
:10540600FF126C882290003AE0FEA3E0FF126C883F
:105416002290003CE0FEA3E0FF126C8822E50D24FA
:1054260088FFE50C3413FE126C88229001FDE0FE25
:10543600A3E0FF126C88229001FBE0FEA3E0FFEFE1
:105446002484FFEE3403FE126C8822AF6FAE6E1218
:105456006C8822E56B2484FFE56A3403FE126C88AF
:1054660022E50B2484FFE50A3403FE126C8822A28F
:105476000FE433FFEF3395E0FEEFC4F8540FC8682E
:10548600FFEEC454F048FEE5A0C4540FFD7C00EFC7
:105496002DFDEE3CFCA210E433FFEF3395E0FEEF6A
:1054A6007805C333CE33CED8F9FFED2FFFEC3EFEA1
:1054B600126C8822900012E0FFEF3395E0FE126C2A
:1054C6008822900013E0FFEF3395E0FE126C8822ED
:1054D600900014E0FFEF3395E0FE126C88229000F6
:1054E60015E0FFEF3395E0FE126C8822900016E07F
:1054F600FFEF3395E0FE126C8822900017E0FFEF75
:075506003395E0FE126C88F2
:01550D00227B
:1068D8009001F0E4F0A3E4F09001F6E4F09001F602
:1068E800E0FFD3EF6480948340030269749001F25F
:1068F800122034000186A020983E9001F2E0FCA30B
:10690800E0FDA3E0FEA3E0FFEC4D4E4F602A9001AE
:10691800F2E0FCA3E0FDA3E0FEA3E0FF7BFF7AFF2B
:1069280079FF78FFEF2BFFEE3AFEED39FDEC38FCEE
:106938009001F212202880BFC2989001F0E0FEA3D7
:10694800E0FF7C007D0A121ECAAD997C00EF2DFF86
:10695800EE3CFEEF24D0FFEE34FFFE9001F0EEF0A7
:10696800A3EFF09001F6E004F00268E59001F0E092
:04697800FEA3E0FF9B
:01697C0022F8
:10570A00900203122034000186A020983E900203E2
:10571A00E0FCA3E0FDA3E0FEA3E0FFEC4D4E4F60EA
:10572A002A900203E0FCA3E0FDA3E0FEA3E0FF7BD6
:10573A00FF7AFF79FF78FFEF2BFFEE3AFEED39FD96
:10574A00EC38FC90020312202880BFC298AF99EF70
:10575A0012208557A36157B26257C16357D0645765
:10576A00DF6557EE6657FD67580C68581B69582A5B
:10577A006A58396B58486C58576D586672586B732B
:10578A00586E74587475588076588C77589878582B
:10579A00A47958B07A000058BB1268D8900024EE59
:1057AA00F0A3EFF0125199221268D8900026EEF079
:1057BA00A3EFF0125199221268D8900028EEF0A3B4
:1057CA00EFF0125199221268D890002AEEF0A3EF56
:1057DA00F0125199221268D890002CEEF0A3EFF043
:1057EA00125199221268D890002EEEF0A3EFF0120F
:1057FA005199221268D8900030EEF0A3EFF01251BE
:10580A0099221268D8900032EEF0A3EFF012519963
:10581A00221268D8900034EEF0A3EFF012519922C8
:10582A001268D8900036EEF0A3EFF01251992212C6
:10583A0068D8900038EEF0A3EFF01251992212685E
:10584A00D890003AEEF0A3EFF0125199221268D8DC
:10585A0090003CEEF0A3EFF012519922D20DD21132
:10586A0022D21122A20FB3920F221268D8900012EC
:10587A00EFF0125095221268D8900013EFF01250F0
:10588A0095221268D8900014EFF0125095221268EF
:10589A00D8900015EFF0125095221268D890001691
:1058AA00EFF0125095221268D8900017EFF01250BC
:0158BA009558
:0158BB0022CA
:10187600021C3CE86480F8E933E83360110460F048
:10188600ED33EC337009E8FCE9FDEAFEEBFF2204D8
:1018960060DED3EB9FEA9EE99DE8C2E78CF0C2F7D3
:1018A60095F0400CE8CCF8E9CDF9EACEFAEBCFFB9F
:1018B600121C0785D0F05804700320D5B3E80470D5
:1018C600075002B2D5021C4692D5EC0460F7E4CC70
:1018D600C0E0C398F8603B94186008400DD0E0FB68
:1018E600021C1EE4FBFAC9FC8028E830E406E4C9C1
:1018F600FBE4CAFCE830E305E4C9CACBFCE85407BC
:101906006010F8C3E913F9EA13FAEB13FBEC13FCC6
:10191600D8F130F52FC3E49CFCEF9BFFEE9AFEED69
:1019260099FDD0E0FBEF4E4D4C701222DB03021CFA
:1019360043EC2CFCEF33FFEE33FEED33FDED30E7E9
:10194600EB021C1EEF2BFFEE3AFEED39FDD0E0FB5D
:1019560050130BBB0003021C46ED13FDEE13FEEF06
:0819660013FFEC13FC021C1E30
:10196E00EC4D6011E8497017ED33EC3304600DE473
:10197E00FCFFFEFD22E933E8330470F8021C3C1232
:10198E001C0758046009E4CC248150062850090233
:10199E001C46284003021C43C0E0EB4A7044B98049
:1019AE0006D0E0FB021C32EF4E701CBD8008EBFF30
:1019BE00EAFEE9FD80EBE98DF0A4FEE5F0021A5790
:1019CE00E9CDF9EAFEEBFFEF89F0A4FCE5F0CE8954
:1019DE00F0A42EFFE435F0CD89F0A42DFEE435F011
:1019EE008067EF4E7005BD80D780C3EF8BF0A4AC3F
:1019FE00F0EE8BF0A42CFCE435F0F8EF8AF0A42C7A
:101A0E00E5F038FCE433CB8DF0A42CFCE5F03BF88C
:101A1E00EE8AF0A42CFCE5F038F8E433CF89F0A47C
:101A2E002CFCE5F038CF3400CE89F0A42FFFE5F082
:101A3E003EFEE433C98DF0A42EFEE5F039CD8AF0DA
:101A4E00A42FFFE5F03EFEE43DFD33D0E0FB500752
:101A5E000BBB000F021C46EC2CFCEF33FFEE33FEEB
:061A6E00ED33FD021C1E19
:101A7400021C46EC5D046005E859047003021C3C3A
:101A8400121C07580460F6EC4860F2EC7004FDFE8A
:101A9400FF22C860DB2481C85009C3986002500645
:101AA400021C439850CAF582E9294B4A7005AB825F
:101AB400021C3275F0007C1A7880C3EF9BEE9AED1D
:101AC40099400DC3EF9BFFEE9AFEED99FDE842F0BD
:101AD400DC23ACF0D0E0FFD0E0FED0E0FDAB822010
:101AE400E7101BEB60BAEC2CFCEF33FFEE33FEED9A
:101AF40033FD021C1EE803F830E705C0F075F00062
:101B0400EF2FFFEE33FEED33FD40B830E7C280AA7D
:101B140074F8CC6480CCC86480C8F582046043C384
:101B2400EB9FF5F0EA9E42F0E99D42F0E89C45F017
:101B340060305018E5825FFFE582F42B5582FB503C
:101B4400210ABA001D09B90019088016E5825BFB59
:101B5400E582F42F5582FF50090EBE00050DBD002D
:101B6400010CC3EB9FF5F0EA9E42F0E99D42F0E8D8
:0D1B74009C45F06007CC4820E701B3EC224F
:101B8100ED33EC33600A047003BD8004ECB2E7FC72
:011B91002231
:101B920075F020800E75F010800575F0087D007ECE
:101BA200007F003392D530D503121F77EC334010FB
:101BB200EF33FFEE33FEED33FDEC33FCD5F0ED22D7
:0E1BC200E5F0247EA2D513CC92E7CDCEFF2213
:101BD000EDD2E7CD33EC3392D524814006E4FFFE0D
:101BE000FDFC22FCE4CFCECDCC24E0501174FF806C
:101BF000EDC3CC13CCCD13CDCE13CECF13CF047009
:071C0000F030D5DE021F7772
:10425000E57B24F5F582E43400F583E0057B2290CC
:1042600000F23009039000F5E475F00112206502B8
:104270001E722002E97F2ED2028018EF540F249084
:10428000D43440D4FF30060BEF24BFB41A005003DF
:104290002461FFE57C6002157C057FE57F700205E7
:1042A0007E30090E9000F2E475F001122065EF02F5
:1042B0001EB8026F217403D2098003E4C209F57BA2
:1042C0009000F212207CE4F57CF57EF57FE57C60C1
:1042D000077F2012429380F5757DFFC203C202C2A0
:1042E00004C205C207C208C20A12425FFF700D3045
:1042F00009057F001242A4AF7FAE7E22B4255FC2C3
:10430000D5C20612425FFF24D0B40A00501A75F0DD
:104310000A787C30D50508B6FF0106C6A426F6202B
:10432000D5047002D20580D924CFB41A00EF50040E
:10433000C2E5D206024596D20380C6D20280C0D220
:104340000480BCD2D580BAD20780B47F20124293B9
:104350002004077401B57C0040F1124250FF124264
:10436000930242CDD20AD2088095124250FB1242EB
:1043700050FA124250F94A4B700679947A467BFF04
:1043800020042EE57C602A7E008E82758300121E3A
:104390008B60060EEE657D70F0C2D5EBC0E0EAC022
:1043A000E0E9C0E0EE1245F7D0E0F9D0E0FAD0E065
:1043B000FB121E72FF60AAEBC0E0EAC0E0E9C0E0B9
:1043C000124293D0E02401F9D0E03400FAD0E0FBAF
:1043D000E57D0460DCD57DD98087D20480A21245BA
:1043E000D960F7E57D700104121C51A97D600DE5CF
:1043F0007D600914F57D124681EF60F3EA30E70233
:10440000F404C3995079EAF4257D0430E701E4040B
:10441000F57D800D1245D960C1EA057D257D121C10
:1044200051EA900121F030E701E4257D04D57D04B7
:10443000200701141245F7E4C0E0124681900121E3
:10444000E0601320E70714F012427B802204F0D0D2
:10445000E014C0E07F0012427BE57D6007124272EB
:10446000157D800B300703124272D0E00242CDD09E
:10447000E00480C41245D9609EE57D04121C519071
:104480000121EAF0E57D20070260010424041245C1
:01449000F734
:1044910074FF04C0E012468112427BE57D200702D1
:1044A1006003124272D0E0B57DE87F4512428590EB
:1044B1000121E07F2B30E7047F2DF404C0E012429C
:1044C10093D0E075F00A84C0F012427CD0E0124231
:1044D1007C0242CD791080027908C208C20A8008A4
:1044E100D2D5790A8004790AC2D5E57D047002F536
:1044F1007DE4FAFDFEFF124250FC7B0820031312FB
:104501004250FD7B1030020A124250FE124250FF0F
:104511007B20EC3382D592D55013C3E43002069F41
:10452100FFE49EFEE42003039DFDE49CFCE4CBF844
:10453100C203EC700CCFCECDCCE824F8F870F38038
:1045410017C3EF33FFEE33FEED33FDEC33FCEB33FA
:10455100FB994002FB0FD8E9EB300305F8D0E0C42A
:1045610048B203C0E00AEC4D4E4F78207B0070C288
:10457100EAB57D0040BCC0E01245F9D0F0D0E020A2
:104581000304C4C0E0C4B203C0F012427CD0F0D531
:10459100F0EB0242CD122085436A5344D558433B88
:1045A1004C43374244D94F44E14444E149435043E9
:1045B10044E75544144644744543DE4746B45043EA
:1045C1003F2D43432E43662B434723436420469D9F
:1045D1002A42FF480000435EE57DB4FF03757D0676
:1045E100124250FC124250FD124250FE124250FF44
:1045F10090011A021C8E790AA2D5200514300709F0
:10460100B910020404B9080104A2D520080250011E
:10461100042004689204B57C005034C0E07F20304F
:1046210005197F30A20472087207500F124650C25A
:1046310004C208C207C20A7F30800F300703E9C0F5
:10464100E0124293300703D0E0F9D0E0B57CCC30E2
:1046510007177F30B9100C1242937F583006077F3D
:10466100788003B908031242933004057F2D02427A
:10467100937F20200AF87F2B2008F322920480CF19
:104681007F00B40700500B241AF582E43401F5834E
:10469100E0FF22286E756C6C2900D2031242503063
:1046A10003F8C203787C30D50108F60242FF2D5091
:1046B1004349581242502403B405004001E4904696
:1046C100AF93124284743A124284D205757C04027B
:0246D10044D5CE
:0D6FD800ED33EC3360065004EC6480FC22C5
:10682C00021C3C22EDA2E7D2E7F9EC3340F260F314
:10683C00B4FF08ED547F70E8021C46F82481C2E0D6
:10684C00C0E0F40428FAC313FCED92E7FD9000E6D7
:10685C00122028EEA2E7E9BA7F02C3133400940099
:10686C00FA75F091A4E5F013F494FE8AF0A433E5E4
:10687C00F033248CD313FDE492E7FE7F007C3F754C
:10688C008302ECC0E0F8EDC0E0F9EEC0E0FAEFC036
:10689C00E0FB8583F09000E6121FD085F083121A7E
:1068AC0077D0E0FBD0E0FAD0E0F9D0E0F812187D18
:1068BC00ED6480FD30E7011CD583C7ED33CC33F894
:0C68CC00D0E0A2E71328C313CC13FD2278
:106ABC009000E61220289000EAE0F8A3E0F9A3E0A9
:106ACC00FAA3E0FB9000E6E0FCA3E0FDA3E0FEA34C
:106ADC00E0FF121A77125C089000E6122028900052
:106AEC00EAE030E7599000E6E0FCA3E0FDA3E0FE0D
:106AFC00A3E0FFECC0E0EDC0E0EEC0E0EFC0E0E4EE
:106B0C00FFFEFDFC9000E6E0F8A3E0F9A3E0FAA399
:106B1C00E0FB121B147BDB600250087A0F7949787A
:106B2C004080067A0F794978C0D0E0FFD0E0FED0E3
:106B3C00E0FDD0E0FC12187D9000E61220289000B9
:0D6B4C00E6E0FCA3E0FDA3E0FEA3E0FF22D5
:105A60003A70FA83BCAAE9E43E81E0F8BF9DE9E61A
:105A70003F80000039283C1ABB9969663DA335E395
:105A8000BF255DE73FC90FDB418DDBCCC44936EE56
:105A900045C9913FC5B0F83D3F800000C317F534BC
:105AA000452FFA73C60AFDDD125B6904A2E192007C
:105AB0001420E015905A607404121D938030125B1C
:105AC0006930E102B20020E0EBA883A9829000E6F1
:105AD00012202889828883905A747404121D938539
:105AE00082F09000E6121FEC85F08212196EED4CE8
:105AF0006007300004EC6480FC22125B69C0E0A8FF
:105B000083A9829000E612202889828883905A987F
:105B10007403121D938582F09000E6121FEC85F04D
:105B20008212196E9000E6E0CCF0A3E0CDF0A3E085
:105B3000CEF0A3E0CFF0905A887403121D93D08268
:105B40008582F09000E6121FEC85F082E58230E05D
:105B500007121A77B2008096EFCBFFEECAFEEDC9AE
:105B6000FDECC8FC121A778085ED33EC547FCC3302
:105B7000920024605007D0E0D0E0021C3C7B837A86
:105B8000F97922783E12196EEDF933ECF83324815D
:105B90005011EFFBEEFA121BD0121B92ECB2E7FC95
:105BA00012187DED33EC33602F2403F8C313FCEDA2
:105BB00092E7FDE82481E4501FECF8EDF9EEFAEFEE
:105BC000FB121BD0EF04C2E0FCF582121B9CECB26E
:105BD000E7FC12187DE58203FAED33EC336007141D
:085BE00013FCED92E7FDEA223F
:105BE800BE1249253E4CCCCDBEAAAAAB3F800000D0
:105BF8003E7ADBB03EED63383F24BC7D3F490FDB86
:105C0800ED33ECC2E7CC339200B4FF13ED547F6060
:105C180003021C3C7FDB7E0F7DC97C3F025CFDC21A
:105C280001C3947F401E7007EDD2E794904015EFB2
:105C3800FBEEFAEDF9ECF87F007E007D807C3F12E8
:105C48001A77D201ED33EC33248430E705E4C0E061
:105C5800806B04FAEDD2E754F0C333DAFD5407340D
:105C6800002323C0E0CCC0E0F8EDC0E0F9EEC0E0CE
:105C7800FAEFC0E0FBE4121B9CEC24FEFC9000EE63
:105C880012202812196E7B007A007980783F12184A
:105C98007D9000EEE0B2E7CCF0A3E0CDF0A3E0CE3B
:105CA800F0A3E0CFF0D0E0FBD0E0FAD0E0F9D0E00C
:105CB800F812187D9000EE121FEC121A779000EE81
:105CC800122028905BE87403121D939000EE121FB7
:105CD800EC12196ED0E0600F24F4F582E4345BF521
:105CE80083121FF812187D30010B7BDB7A0F79C9FC
:105CF80078BF12187DED33EC336006ECA20092E712
:025D0800FC227B
:10636E009000E612202874FFFFFEFDFC9000E6E090
:10637E00F8A3E0F9A3E0FAA3E0FBC3121F8560388F
:10638E007F807E967D187C4B9000E6E0F8A3E0F9C6
:10639E00A3E0FAA3E0FB121B146002501B7F807E69
:1063AE00967D187CCB9000E6E0F8A3E0F9A3E0FA26
:1063BE00A3E0FB121B14500F9000E6E0FCA3E0FDDF
:1063CE00A3E0FEA3E0FF229000E6E0FCA3E0FDA325
:1063DE00E0FEA3E0FF121BD09000EA1220289000EE
:1063EE00EAE0FCA3E0FDA3E0FEA3E0FFEC121B92AB
:1063FE00C8ECC8C9EDC9CAEECACBEFCB9000E6E037
:10640E00FCA3E0FDA3E0FEA3E0FF121879E4FBFA83
:10641E00F9F8121B14602640249000EAE0FCA3E079
:10642E00FDA3E0FEA3E0FFEF24FFFFEE34FFFEED41
:10643E0034FFFDEC34FFFC9000EA1220289000EAB5
:10644E00E0FCA3E0FDA3E0FEA3E0FFEC121B922212
:101C0700E9D2E7C933E833F892D5EDD2E7CD33EC23
:071C170033FC5002B2D5229C
:101C1E00EC30E7100FBF000C0EBE00080DBD000427
:101C2E000BEB6014A2D5EB13FCED92E7FD2274FFD3
:101C3E00FCFDFEFF22E480F8A2D574FF13FC7D802C
:031C4E00E480EF40
:101C5100F920E73624F950037907E4F42402FBE57F
:101C610082158270021583DBF6E024FB501BE960CC
:101C710014E4F0E582158270021583E004F0B40AE1
:0D1C810008E4F0D9EE7401F00A22C2D52269
:101C8E00ED33EC3392D5FA602AB4FF33EDC2E77B25
:101C9E00FF60067A1C79B3E4227A1C79BC20D50445
:101CAE007A1C79B7224E614E002B494E46002D49C3
:101CBE004E4600E47A08F0A3DAFC7B00740722C0DB
:101CCE0083C082ECC0E0EDC0E0EEC0E0EFC0E0EA21
:101CDE0075F010A4CAABF075F04DA42BFBE435F0F3
:101CEE00FCEA2410FAEB34C5FBEC34D9FCEDC2E768
:101CFE00FF75F056A4F42411C5F0F434C58FF0A48A
:101D0E002AE5F03BE43CF020E714121E10D0E0FF71
:101D1E00D0E0FED0E0FDD0E0FC121A778014F4047F
:101D2E00121E10D0E0FFD0E0FED0E0FDD0E0FC129D
:101D3E00196ED082D083E0FAEDD2E7CD33EC3324A6
:101D4E0082FBE4C3CF33CFCE33CECD33CD33DBF3F3
:101D5E007B0775F00A846004F0A31B0AE5F0F0A37C
:101D6E008FF0740AA4FFACF08EF0740AA42CFEACB3
:101D7E00F050010C8DF0740AA42CFDE435F0F0A3A4
:051D8E00DBDE740722FA
:101D9300C0E0EFFBEEFAEDF9ECF812196ED0E0F5C6
:101DA300F0EFFBEEFAEDF9ECF8121FDCA3A3A3A30B
:101DB300E8C0E0E9C0E0EAC0E0EBC0E0C0F012191F
:101DC3006E121FF8A3A3A3A312187DD0F0D0E0FBDB
:0D1DD300D0E0FAD0E0F9D0E0F8D5F0D4224D
:101DE0003F8000004120000042C80000447A00000B
:101DF000461C400047C35000497424004B1896808D
:101E00004CBEBC205A0E1BCA6753C21C749DC5AE83
:101E1000FB60065407601C2323121E3EEB543860FF
:101E200009121E2A121E3912196EECF8EDF9EEFA9B
:101E3000EFCB22EB121E3980F1543803241C901D85
:101E4000E0FE93FC0EEE93FD0EEE930ECE93FF227A
:106A3C00022245E493A3F8E493A34003F68001F209
:106A4C0008DFF48029E493A3F85407240CC8C3335B
:106A5C00C4540F4420C8834004F456800146F6DF2A
:106A6C00E4800B0102040810204080906E12E47E3A
:106A7C00019360BCA3FF543F30E509541FFEE4931F
:106A8C00A360010ECF54C025E060A840B8E493A3E6
:106A9C00FAE493A3F8E493A3C8C582C8CAC583CA11
:106AAC00F0A3C8C582C8CAC583CADFE9DEE780BEC9
:016E5A000037
:101E5000C2D530F707B2D563F0FF05F030E70CB21A
:101E6000D5F4048463F0FF05F080018430D502F4DA
:021E700004224A
:101E7200BB010689828A83E0225002E722BBFE026E
:091E8200E32289828A83E49322A1
:101E8B00BB010CE58229F582E5833AF583E022500C
:101E9B0006E92582F8E622BBFE06E92582F8E22256
:0D1EAB00E58229F582E5833AF583E4932270
:101EB800BB010689828A83F0225002F722BBFE0109
:021EC800F32203
:101ECA00EF8DF0A4A8F0CF8CF0A428CE8DF0A42E2C
:021EDA00FE22E6
:101EDC00C2D5EC30E709B2D5E4C39DFDE49CFCEE21
:101EEC0030E715B2D5E4C39FFFE49EFE1220D8C3A1
:101EFC00E49DFDE49CFC80031220D830D507C3E49C
:061F0C009FFFE49EFE228F
:101F1200C5F0F8A3E028F0C5F0F8E582158270025A
:061F22001583E038F022F7
:101F2800E88FF0A4CC8BF0A42CFCE98EF0A42CFC58
:101F38008AF0EDA42CFCEA8EF0A4CDA8F08BF0A4D6
:101F48002DCC3825F0FDE98FF0A42CCD35F0FCEB35
:101F58008EF0A4FEA9F0EB8FF0A4CFC5F02ECD39FA
:0F1F6800FEE43CFCEAA42DCE35F0FDE43CFC2267
:106E5B00C2D5E830E70FB2D5E4C39BFBE49AFAE462
:106E6B0099F9E498F8EC30E717B2D5126E9112212C
:106E7B0069E4C39BFBE49AFAE499F9E498F880037C
:106E8B0012216930D50DE4C39FFFE49EFEE49DFD06
:046E9B00E49CFC2255
:0E1F7700C3E49FFFE49EFEE49DFDE49CFC227B
:101F8500EB9FF5F0EA9E42F0E99D42F0E89C45F0B2
:011F95002229
:101F9600BB010789828A83021FD05005E9F8022116
:101FA600FBBBFE05E9F802220789828A83021FDC51
:101FB600BB010789828A830220285005E9F802229C
:0A1FC6002DBBFE05E9F802223922C6
:0C1FD000E0FCA3E0FDA3E0FEA3E0FF2284
:101FDC00E493FC740193FD740293FE740393FF224B
:0C1FEC00E0F8A3E0F9A3E0FAA3E0FB2278
:101FF800E493F8740193F9740293FA740393FB223F
:10200800BB010789828A83021FEC5005E9F8022286
:1020180013BBFE05E9F802222089828A83021FF891
:0C202800ECF0A3EDF0A3EEF0A3EFF0222B
:10203400A8828583F0D083D08212204B12204B12C9
:10204400204B12204BE473E493A3C583C5F0C583EE
:10205400C8C582C8F0A3C583C5F0C583C8C582C8F6
:012064002259
:10206500F8E0FBA3A3E0F925F0F0E5821582700204
:072075001583E0FA38F022A8
:09207C00EBF0A3EAF0A3E9F02265
:10208500D083D082F8E4937012740193700DA3A3EA
:1020950093F8740193F5828883E4737402936860FE
:0620A500EFA3A3A380DFFE
:1020AB00D083D082F8E4937012740193700DA3A3C4
:1020BB0093F8740193F5828883E473740293B5F0FB
:0D20CB00067403936860E9A3A3A3A380D863
:106F2100EFB40A07740D126F2C740A309811A899E6
:106F3100B8130CC2983098FDA899C298B811F630D0
:076F410099FDC299F59922A8
:106F6000C3EE6480948040028007C3E49FFFE49EE8
:026F7000FE22FF
:1020D800BC000BBE0029EF8DF084FFADF022E4CCEC
:1020E800F875F008EF2FFFEE33FEEC33FCEE9DECB5
:1020F800984005FCEE9DFE0FD5F0E9E4CEFD22EDFB
:10210800F8F5F0EE8420D21CFEADF075F008EF2F44
:10211800FFED33FD4007985006D5F0F222C398FD35
:052128000FD5F0EA22D2
:10212D0075F008758200EF2FFFEE33FECD33CDCC69
:10213D0033CCC58233C5829BED9AEC99E5829840EC
:10214D000CF582EE9BFEED9AFDEC99FC0FD5F0D6C9
:10215D00E4CEFBE4CDFAE4CCF9A88222B800C1B9F3
:10216D000059BA002DEC8BF084CFCECDFCE5F0CB31
:10217D00F97818EF2FFFEE33FEED33FDEC33FCEB6A
:10218D0033FB10D703994004EB99FB0FD8E5E4F925
:10219D00FA227818EF2FFFEE33FEED33FDEC33FC12
:1021AD00C933C910D7059BE99A4007EC9BFCE99A06
:1021BD00F90FD8E0E4C9FAE4CCFB2275F010EF2F4B
:1021CD00FFEE33FEED33FDCC33CCC833C810D7074B
:1021DD009BEC9AE899400AED9BFDEC9AFCE899F886
:0E21ED000FD5F0DAE4CDFBE4CCFAE4C8F92219
:0C21FB00E6FC08E6FD08E6FE08E6FF2210
:0C220700E2FC08E2FD08E2FE08E2FF2213
:0D221300E6FB08E6F908E6FA08E6CBF8223B
:0D222000E2FB08E2F908E2FA08E2CBF8223E
:0C222D00ECF608EDF608EEF608EFF622DD
:0C223900ECF208EDF208EEF208EFF222E1
:00000001FF
